:100000000C948D020C94AA020C94AA020C94AA02DD
:100010000C94AA020C94AA020C94AA020C94AA02B0
:100020000C94AA020C94F70F0C94AA020C94D80F0B
:100030000C94751B0C94AA020C94AA020C94AA02AC
:100040000C94AA020C94AA020C94ED0E0C94AA0231
:100050000C94AE050C94AA020C9478050C94AA0298
:100060000C9487110C94AA020C94861A0C94AA0280
:10007000A31AA81ABC1AC91AD61ACE1AD61AE81A7E
:10008000121BF91AFD1A1D1B071B121B001B041B58
:100090001D1B071B121B161B1A1B1D1B211B0A0AEB
:1000A0000D004E65757472616C0048656164696E1F
:1000B00067486F6C64000A0D537465756572756EE0
:1000C000673A20004F4B0A0D000A0D4162676C65CC
:1000D000696368204C756674647275636B73656ED2
:1000E000736F722E2E000A0D42656E75747A65204C
:1000F000506172616D657465727361747A202564F4
:10010000000A0D414343206E696368742061626791
:1001100065676C696368656E21000A0D496E6974D4
:100120002E20454550524F4D3A2047656E6572610D
:1001300074696E672044656661756C742D506172D8
:10014000616D65746572207573696E67206F6C648C
:1001500020537469636B2053657474696E67730010
:100160000A0D496E69742E20454550524F4D3A2074
:1001700047656E65726174696E6720446566617576
:100180006C742D506172616D6574657220616E646E
:1001900020537469636B2D53657474696E67732E95
:1001A0002E2E000A0D3D3D3D3D3D3D3D3D3D3D3D3D
:1001B0003D3D3D3D3D3D3D3D3D3D3D3D3D3D3D3D6F
:1001C0003D3D3D000A0D466C69676874436F6E746F
:1001D000726F6C0A0D48617264776172653A2564CA
:1001E0002E25640A0D536F6674776172653A562541
:1001F000642E2564256320002E0048693A25346961
:10020000202043663A253469200047733A25346933
:10021000202047693A25346920004E693A2534691F
:100220002020526F3A253469200045787465726E3B
:10023000436F6E74726F6C20200052616E67653A76
:100240002533692D253369005374656C6C756E67B1
:100250003A2025336900536574706F696E742020ED
:1002600025336900536572766F202000506F7469E2
:10027000343A202025336900506F7469333A2020C6
:1002800025336900506F7469323A202025336900A4
:10029000506F7469313A20202533690053746172BC
:1002A000743A2020202020253569004D657373772E
:1002B0006572743A20202535690052696368747547
:1002C0006E673A2020253569004B6F6D706173733E
:1002D0002020202020202000456D70662E5065676C
:1002E000656C3A253569005370616E6E756E673ABC
:1002F000202025356900486F63682025346920284F
:100300002533692900526F6C6C202534692028251B
:10031000336929004E69636B202534692028253311
:10032000692900414343202D2053656E736F72008D
:1003300047696572202534692028253369292825D5
:1003400033692900526F6C6C2025346920282533CD
:1003500069292825336929004E69636B2025346992
:1003600020282533692928253369290047696572C2
:100370002025346920282533692900526F6C6C20B0
:10038000253469202825336929004E69636B2025AF
:10039000346920282533692900476965722025348E
:1003A0006920282533692900526F6C6C2025346937
:1003B000202825336929004E69636B202534692084
:1003C0002825336929004779726F202D2053656EE7
:1003D000736F720050333A253469202050343A2527
:1003E0003469200050313A253469202050323A25B2
:1003F0003469200047733A253469202047693A253B
:10040000346920004E693A2534692020526F3A251C
:10041000346920004B373A25346920204B383A257F
:10042000346920004B353A25346920204B363A2573
:10043000346920004B333A25346920204B343A2567
:10044000346920004B313A25346920204B323A255B
:10045000346920004B6F6D706173733A2020202542
:10046000356900526F6C6C3A202020202020253501
:1004700069004E69636B3A202020202020253569D1
:1004800000616B742E204C6167650048F668656EEC
:10049000726567656C756E67004B65696E652000F7
:1004A0004F66662020202020203A20253569004C08
:1004B000756674647275636B3A2025356900526500
:1004C000674F66667365743A20253569002863298D
:1004D00020486F6C676572204275737300536574B2
:1004E00074696E673A202564200048573A5625649F
:1004F0002E25642053573A25642E25642563002B4E
:10050000204D696B726F4B6F70746572202B005BAE
:1005100025695D005B25695D000011241FBECFEFDA
:10052000D0E1DEBFCDBF14E0A0E0B1E0E0EFF7E93D
:1005300002C005900D92AC3BB107D9F719E0ACEBC6
:10054000B4E001C01D92A73AB107E1F70E943B0356
:100550000C94F74B0C940000863010F085E002C03C
:10056000882329F0A2E0B0E0082E0E94EB4B08950A
:10057000A2E0B0E00E94E34B902D892F815085309E
:1005800020F083E00E94AC0293E0892F90E0089570
:1005900080919C08E82FF0E0EE0FFF1FE259F74F23
:1005A000808191818D5E9F4F14F0109202018081B5
:1005B00091818A5B9F4FBCF480910201882399F45A
:1005C00081E08093020180916B078F5F80936B07BE
:1005D000853038F088EE93E09093DE048093DD045C
:1005E00002C00E94912880916B0790E09093390897
:1005F000809338080895582FFB01863010F055E09D
:1006000002C08823D1F0252F30E021503040842FC4
:1006100090E0289FD001299FB00D389FB00D112484
:10062000AC59BF4F019724F001900E94EB4BFACFD9
:10063000852F0E94AC020E942B430895282FFB01B6
:100640008150853008F023E030E021503040842F85
:1006500090E0289FD001299FB00D389FB00D112444
:10066000AC59BF4F019724F00E94E34B0192FACF9F
:100670000E942B4308951F93CF93DF9314B815B8AE
:10068000189B06C0199B02C08DE007C08BE005C017
:10069000199B02C084E101C08AE08093000181E8D7
:1006A00087B93E9A8FEF88B98BE184B981E085B92B
:1006B0008EE38AB9579A87E78BB984B7877F84BF5F
:1006C000809160008861809360001092600080EDEE
:1006D00097E09093DE048093DD04109280051092E1
:1006E0007F05109273081092720810927E05109286
:1006F0007D0510927C0510927B05809100018A3067
:1007000011F0843111F4289801C0289A0E94231115
:100710000E941D070E94601B0E9481110E946C1A9A
:100720000E941440789420910001822F6AE00E9478
:100730003C4B492F50E0822F0E943C4B90E022E638
:1007400030E03F932F932AE030E03F932F9321E056
:1007500030E03F932F935F934F939F938F9384EC5D
:1007600091E09F938F931F920E94490C83EA91E03E
:100770009F938F931F920E94490C8DB79EB740960E
:100780000FB6F8949EBF0FBE8DBF809100018C30D4
:1007900010F4299A01C0299849E06CE978E083E0D7
:1007A0000E941E0321E030E0D9010E94E34B802D1E
:1007B0008F3FB1F0D9010E94E34B802D893480F046
:1007C00080919C088A3060F480919D088A3040F4C2
:1007D00080919E088A3020F480919F088A3050F0E2
:1007E00080E691E09F938F931F920E94490C0E9494
:1007F000511C0DC0D9010E94E34B802D893451F06A
:100800008AE191E09F938F931F920E94490C0F9071
:100810000F900F90A1E0B0E00E94E34B802D89344F
:1008200009F10E94EC2911E0CCE9D8E0123039F04E
:10083000133019F40E94A62804C0143010F00E944E
:10084000482946E5BE01812F0E94FB021F5F16303A
:1008500069F783E00E94AC0289E4A1E0B0E0082ED1
:100860000E94EB4BA4E0B0E00E94E34B802D85306A
:1008700050F081E091E09F938F931F920E94490C6A
:100880000F900F900F900E94B80246E56CE978E057
:100890000E941E030E94B80290E09F938F9386EE01
:1008A00090E09F938F931F920E94490C8091A4081F
:1008B0000F900F900F900F900F9080FD03C0C8EE27
:1008C000D3E020C089EC90E09F938F931F920E9409
:1008D000490C88EE93E00E94C30FEC010E94EC14D7
:1008E0000F900F900F90CE010E94CC0F8823D9F368
:1008F00084EC90E09F938F931F920E94490C0F907D
:100900000F900F900E94EA26809100018A3011F02A
:10091000843111F4289801C0289A80ED97E09093D3
:10092000DE048093DD0485E580936D0786EB90E01F
:100930009F938F931F920E94490C8091A4080F905F
:100940000F900F9082FF03C08AEA90E002C082EA13
:1009500090E09F938F931F920E94490C0F900F90ED
:100960000F908EE990E09F938F931F920E94490C05
:100970000E94371588E893E1909392038093910346
:1009800081E080936C070F900F900F908091DA04B4
:10099000882309F4A5C01092DA0480916B0788239C
:1009A00019F00E94C80202C00E948E2A0E943C25B3
:1009B000209100012A3011F0243111F4289801C04F
:1009C000289A80910501882321F0815080930501A8
:1009D0000EC01092770710929D0510929C05109200
:1009E0009F0510929E051092A1051092A00580917E
:1009F0007A05882329F080917A05815080937A05C1
:100A00008091910390919203892B01F585E090E00C
:100A100090939203809391030E943A1B80910B0361
:100A200090910C038F5F9F4F09F580918305882378
:100A3000E9F080E197E29093DE048093DD0480E8A2
:100A400090E090930C0380930B0310C0809191036E
:100A500090919203019790939203809391032A308F
:100A600011F0243111F4289801C0289A8091DA04F9
:100A7000882321F080918305882311F40E942A089D
:100A80000E94F109CE010E94CC0F882339F12091F8
:100A90001103309112038091B40890E028173907B0
:100AA0009CF480910B0390910C038F5F9F4F61F436
:100AB00080E797E19093DE048093DD0480E093E08B
:100AC00090930C0380930B030E94404284E0809338
:100AD000DF0484E190E00E94C30FEC010E943E43DA
:100AE0008091DF04882309F051CF0E9481424ECFCC
:100AF0001F920F920FB60F9211248F939F93EF9333
:100B0000FF93809103018823E1F48091D6049091B2
:100B1000D70401969093D7048093D604FC01E35D3B
:100B2000F94FE081ED3019F08639910539F41092D2
:100B3000D7041092D60481E080930301E093C600AD
:100B400004C01092D7041092D604FF91EF919F91A8
:100B50008F910F900FBE0F901F9018951F920F92BC
:100B60000FB60F9211242F933F934F938F939F9320
:100B7000AF93BF93CF93DF93EF93FF938091C60022
:100B80008093C3044091D104463910F01092D004F0
:100B90008091C3048D3009F05DC08091D004823013
:100BA00009F058C01092D004A42FB0E0FD01E8581D
:100BB000F84F3081ED01C758D84F28818091D40477
:100BC0009091D504831B9109821B91099F7090938A
:100BD000D5048093D4049C0196E0369527959A9588
:100BE000E1F7235C2093D304982F9F73935C909339
:100BF000D2048081281729F48881981711F491E094
:100C000006C08091C6048F5F8093C60490E08091F7
:100C1000C404882309F066C0992309F463C081E005
:100C20008093C4044F5F4093C704A658B84F8DE02B
:100C30008C9380917C07823509F054C088E190E064
:100C40002CE00FB6F894A895809360000FBE209317
:100C5000600048C08091D0048130D9F0813018F014
:100C60008230F1F521C08091C304833239F4809140
:100C7000C404882319F481E08093D0048091C304D4
:100C800080937A0781E08093D1048091C30490E03F
:100C900022C082E08093D004E42FF0E08091C3046E
:100CA000E658F84F808309C0E42FF0E08091C30438
:100CB000E658F84F8083463920F44F5F4093D104C3
:100CC00002C01092D0042091C3048091D40490916A
:100CD000D504820F911D9093D5048093D40402C053
:100CE0001092D004FF91EF91DF91CF91BF91AF911E
:100CF0009F918F914F913F912F910F900FBE0F9029
:100D00001F901895DC0120E030E040E050E008C082
:100D1000FA01E35DF94F8081280F311D4F5F5F4F6E
:100D20004A175B07A9F73F70C90136E0969587958A
:100D30003A95E1F7835CFD01E35DF94F80831196FD
:100D40002F73235CFD01E35DF94F2083A25DB94F52
:100D50008DE08C931092030180912D068093C60044
:100D600008953091C704365043E063E046C0E42F55
:100D7000F0E0E658F84F80814F5FE42FF0E0E6584E
:100D8000F84F20814F5FE42FF0E0E658F84F708174
:100D90004F5FE42FF0E04350E658F84F50812D5359
:100DA000E62FF0E0922F92959F708D53880F880F59
:100DB000892BE658F84F8083E62FEF5F313009F139
:100DC000972F9D53F0E02295207F892F8695869559
:100DD000282BE658F84F2083E62FEE5F33503F3F35
:100DE00081F04C5FF0E09295990F990F907C5D53E4
:100DF000952BE658F84F90836D5F332309F0B7CFFA
:100E0000E62F8DE797E09093C9048093C804E350E0
:100E1000E093CA0408951F93182F8A3019F48DE0C7
:100E20000E940B078091C00085FFFCCF1093C60085
:100E300080E090E01F9108950895E1ECF0E088E1F2
:100E40008083A0ECB0E08C9182608C93808180687C
:100E500080838081806480838AE28093C400809153
:100E60000701909108010E94C30F90935A07809345
:100E700059078CED90E00E94C30F909379078093FF
:100E8000780791E090935B078AE080935C079093EA
:100E90005F0780935D0710925E071092C90410925D
:100EA000C8041092CA040895DF92EF92FF920F9344
:100EB0001F93CF93DF93CDB7DEB722970FB6F89489
:100EC000DEBF0FBECDBF9D85AE8583E280932D062C
:100ED0009F5990932E068C8580932F06CE010F96F6
:100EE0009A838983AA2341F4EE24FF2460E070E012
:100EF00003E010E0B0E094C0EF84F888CE014396A0
:100F00009A83898369897A89A150F2CFF701EB0F1F
:100F1000F11D9081BF5F6150704011F09B0113C0C3
:100F2000AA2309F483C0E981FA81E080F180349634
:100F3000FA83E983349722813381A1502115310549
:100F400009F473C0B0E0F701EB0FF11D4081BF5F02
:100F5000B90161507040A9F4AA2311F4DD2427C01F
:100F6000E981FA81E080F1803496FA83E98334974D
:100F700062817381A1506115710511F4DD2416C0E1
:100F8000B0E0F701EB0FF11DD080BF5F6150704002
:100F900071F4AA2361F0E981FA81E080F18034964E
:100FA000FA83E983349762817381A150B0E0892F7D
:100FB00086958695835CF801E35DF94F808350E068
:100FC0009A0184E0369527958A95E1F7892F90E07C
:100FD00083709070F4E0880F991FFA95E1F7282B41
:100FE000235CF801E25DF94F20838D2D8295869573
:100FF000869583704F705070440F551F440F551FD6
:10100000842B835CF801E15DF94F80838FE3D82264
:101010008DE3D80EF801E05DF94FD0820C5F1F4FD1
:101020006115710509F072CF04C0B0E0DD2440E025
:10103000BECFC8010E94820622960FB6F894DEBF8A
:101040000FBECDBFDF91CF911F910F91FF90EF9019
:10105000DF90089580910301882309F4C1C1809134
:10106000BE048823C1F1809103018823A1F10E946D
:1010700040158091C20424E1829FC00111248A5D41
:101080009C4F24E130E03F932F939F938F9381E017
:1010900090E09F938F9382EC94E09F938F9382E0F4
:1010A0008F9381E08F9388E48F930E9454078091FF
:1010B000C2048F5F8093C2042DB73EB7255F3F4FB8
:1010C0000FB6F8943EBF0FBE2DBF843010F01092C3
:1010D000C2041092BE048091BD04882371F18091F6
:1010E0000301882351F10E94401580E590E09F9311
:1010F0008F9386E293E09F938F9321E030E03F93BC
:101100002F9386E793E09F938F933F932F938CE0E9
:1011100095E09F938F9383E08F9381E08F938CE48E
:101120008F930E9454071092BD048DB79EB70F96FF
:101130000FB6F8949EBF0FBE8DBF8091C004882368
:10114000F1F0809103018823D1F08AE090E09F9331
:101150008F938BE597E09F938F9381E08F938F938D
:1011600086E58F930E9454071092C0042DB73EB7B6
:10117000295F3F4F0FB6F8943EBF0FBE2DBF809141
:10118000BC048823F9F0809103018823D9F02091D1
:1011900006018BE090E09F938F938DE697E09F93FD
:1011A0008F9381E08F932F9387E48F930E9454074E
:1011B0001092BC048DB79EB707960FB6F8949EBFE9
:1011C0000FBE8DBF80917807909179070E94CC0F58
:1011D000882309F459C080910301882309F454C07D
:1011E00060912B0570912C0580912D0590912E0515
:1011F0002CE630E040E050E00E94914B30936607CF
:101200002093650760913305709134058091350511
:10121000909136052CE630E040E050E00E94914B82
:101220003093680720936707809192058093690740
:101230008091930580936A0788E090E09F938F9355
:1012400085E697E09F938F9381E08F9383E08F9360
:1012500087E78F930E9454072DB73EB7295F3F4F12
:101260000FB6F8943EBF0FBE2DBF80916B0785303F
:1012700018F086E080936B0783E690E00E94C30F2E
:1012800090937907809378078091070190910801E6
:10129000892B41F08091590790915A070E94CC0FF9
:1012A000882321F48091BF04882351F180910301A8
:1012B000882331F182E490E09F938F9380E198E05E
:1012C0009F938F9381E08F938F9384E48F930E94F9
:1012D00054071092BF0480910701909108012DB727
:1012E0003EB7295F3F4F0FB6F8943EBF0FBE2DBFEC
:1012F000009731F00E94C30F90935A0780935907CB
:10130000809104018F3F49F190E024E0880F991FFC
:101310002A95E1F7875F9E4F20E130E03F932F93BE
:101320009F938F9381E090E09F938F9384E091E06F
:101330009F938F9382E08F9381E08F9381E48F93CB
:101340000E9454078FEF809304018DB79EB70B96D0
:101350000FB6F8949EBF0FBE8DBF809152088823B0
:10136000F1F0809103018823D1F081E090E09F9318
:101370008F9382E598E09F938F9381E08F938F9373
:1013800082E48F930E945407109252082DB73EB703
:10139000295F3F4F0FB6F8943EBF0FBE2DBF80911F
:1013A000C1048823E9F0809103018823C9F086E114
:1013B00090E09F938F938EE698E09F938F9381E0C8
:1013C0008F938F9380E58F930E9454071092C104EE
:1013D0008DB79EB707960FB6F8949EBF0FBE8DBF10
:1013E00008950F931F93CF93DF93CDB7DEB7229766
:1013F0000FB6F894DEBF0FBECDBF8091C404882322
:1014000009F4E3C10E94B10680917B07823609F09E
:101410000DC180917C07813709F448C0823730F4D0
:101420008B3459F0803709F001C13CC0833709F48F
:1014300093C0843709F0FAC021C0E091C804F0914C
:10144000C90480819181909368058093670580919C
:101450006705909168052091690530916A05845E61
:101460009D4F821B930B68E671E00E945C4B845B8E
:10147000904090936C0580936B05D8C0E091C804B0
:10148000F091C90480819181A281B3818093CC04C1
:101490009093CD04A093CE04B093CF048FEF8093AC
:1014A0000501C4C081E08093C104C0C00091C8049C
:1014B0001091C904F80180818F3F21F40E94B80285
:1014C000F8018083E091C804F091C90480818823E9
:1014D00011F481E003C0863010F085E08083E09154
:1014E000C804F091C90446E56CE978E080810E9467
:1014F0001E03809103018823E1F3E091C804F09179
:10150000C9048081898389E48A8386E590E09F937A
:101510008F938CE998E09F938F9321E030E03F9385
:101520002F93CE0102969F938F933F932F93CE01DB
:1015300001969F938F9383E08F9381E08F9381E552
:101540008F930E9454078DB79EB70F960FB6F894ED
:101550009EBF0FBE8DBF6AC0E091C804F091C90460
:1015600080818150853008F045C08181893409F03F
:1015700041C0ACE9B8E0329686E501900D92815009
:10158000E1F7E091C804F091C90446E56CE978E020
:1015900080810E94FB026091C70870E080E090E0CB
:1015A00024EC39E040E050E00E941D4B609395032D
:1015B0007093960380939703909398036091C80863
:1015C00070E080E090E00E941D4B6093990370935F
:1015D0009A0380939B0390939C03E091C804F0913D
:1015E000C90480810E94AC020E94B80289830E94D3
:1015F000912801C01982809103018823E1F381E0E1
:1016000090E09F938F93CE0101969F938F9381E0FB
:101610008F938F9383E58F930E945407EDB7FEB7A6
:1016200037960FB6F894FEBF0FBEEDBF80917C07D2
:10163000873609F4BFC0883680F4813609F460C06B
:10164000823620F48B3409F0B8C039C0823609F4F0
:1016500064C0843609F0B1C073C08C3609F498C0F8
:101660008D3620F4883609F0A8C07DC0843721F07B
:10167000863709F0A2C09AC0E091C804F091C9046D
:1016800080819181A281B3818093CC049093CD0419
:10169000A093CE04B093CF04809103018823E1F39B
:1016A000809106011F928F9384E58F930E945407C7
:1016B0008FEF809305010F900F900F907EC0E09107
:1016C000C804F091C904808191819093680580934A
:1016D00067058091670590916805209169053091B3
:1016E0006A05845E9D4F821B930B68E671E00E9441
:1016F0005C4B845B904090936C0580936B055DC060
:10170000E091C804F091C904808180930401803283
:1017100098F08FE1809304010FC0ADE6B7E0E0914F
:10172000C804F091C9048BE001900D928150E1F75B
:1017300080917607809352088FEF809305013DC01A
:10174000E091C804F091C90480812AE0829FC00121
:1017500011249093080180930701892B71F181E096
:101760008093BF042AC08FEF80930501E091C804E5
:10177000F091C904808190910D05892B80930D050E
:10178000882311F01092C20481E08093BE0415C03A
:101790008FEF80930501E091C804F091C904808126
:1017A00080930C0581E08093BD0407C081E08093A5
:1017B000C00403C081E08093BC041092C404109262
:1017C000C9041092C8041092CA0422960FB6F89465
:1017D000DEBF0FBECDBFDF91CF911F910F91089556
:1017E000982F80915308813069F480910B05E82F80
:1017F000F0E0EA5DFC4F90838F5F80930B0521E062
:1018000030E005C0892F0E940B07282F30E0C90166
:1018100008951F93182F04C080E30E94F00B11500D
:101820001116D4F31F9108951F93182F04C080E25E
:101830000E94F00B11501116D4F31F9108950F93CD
:101840001F93CF93DF938C01EB0108C0F8010F5F6A
:101850001F4FE4918E2F0E94F00B21972097B1F734
:10186000DF91CF911F910F9108950F931F93CF9305
:10187000DF938C01EB0106C0F80181918F010E947A
:10188000F00B21972097C1F7DF91CF911F910F9116
:1018900008952F923F924F925F926F927F928F9214
:1018A0009F92AF92BF92CF92DF92EF92FF920F93EF
:1018B0001F93CF93DF93CDB7DEB7E5970FB6F894BC
:1018C000DEBF0FBECDBF2B968FAD2B9780935308F5
:1018D000CE01835B9F4F9B838A832D964EAC5FAC7A
:1018E0002D971EA61FA618AA19AA9E01225D3F4F7A
:1018F0003DAB2CAB820102C00F5F1F4FF801F4908B
:10190000FF2019F0F5E2FF16B9F7B801641975095F
:1019100019F0C2010E941F0CFF2009F445C22801E2
:101920000894411C511C1982AA81BB8133241BAA33
:101930002FEF2AABF2010894411C511CB490632D87
:1019400070E06170707035E7B31621F08B2D806206
:101950008837C9F46115710559F02D913D914D916C
:101960005C9113972EA73FA748AB59AB14960BC0B9
:101970008D919C9111979C0140E050E02EA73FA7CC
:1019800048AB59AB129630E2B31621F48981882313
:1019900089F61CC043E2B41611F458E055C08AE23F
:1019A000B81621F09DE2B91671F408C0FD01129637
:1019B000E081EBABE7FFBECFE195EBABE0E13E2A88
:1019C000FFED3F22B7CF2BE2B21611F4B982B2CFAE
:1019D0003EE2B31699F5F2010894411C511C849122
:1019E0008A3221F0B82E20E030E01DC0FD011296B1
:1019F0004081518157FF02C04FEF5FEF4AAB9ACF52
:101A0000C90153E0880F991F5A95E1F7220F331F40
:101A1000280F391F2B0D311D20533040F20108943F
:101A2000411C511CB4908B2D80538A3048F3A9017E
:101A300037FF02C04FEF5FEF4AAB85CF40E3B416EC
:101A400029F434FC77CF50E2352A74CF8B2D8153A3
:101A50008930D8F420E030E0C90103E0880F991FF5
:101A60000A95E1F7220F331F280F391F2B0D311D67
:101A700020533040F2010894411C511CB4908B2D2E
:101A800080538A3048F32BAB5ECF88E6B81619F442
:101A900094E0392A4FCFECE6BE1619F4F1E03F2A64
:101AA00049CFBB83AA8323E6B21639F41296BB83CF
:101AB000AA8312978C918E8322C134E4B31639F035
:101AC00044E6B41631F059E6B516A9F502C081E036
:101AD000382A30FE08C01496BB83AA835E914E91CB
:101AE0003E912E910AC01296BB83AA839E918E913D
:101AF0009C01442737FD4095542F2EA73FA748ABA4
:101B000059AB8EA59FA5A8A9B9A9BB238CF42EA576
:101B10003FA548A959A950954095309521953F4F2B
:101B20004F4F5F4F2EA73FA748AB59AB8DE289833C
:101B3000BAE02B2E80C03FE4B31621F04FE6B41676
:101B400031F402C051E0352AA8E02A2E73C080E7A4
:101B5000B81689F41296BB83AA839E918E919C013C
:101B600040E050E02EA73FA748AB59AB30E4332A02
:101B7000F8E7BF2E5DC043E7B416D1F51296BB83DC
:101B8000AA83DE90CE90C114D10489F488E28E83BA
:101B90008EE68F8385E788878CE689878A8789E246
:101BA0008B871C86E6E0CE2ED12CCC0EDD1E5AA9EA
:101BB00057FD14C0452F552747FD509560E070E054
:101BC000C6010E94F548009711F4FAA80EC0F82E3D
:101BD000FC188AA98F154CF4F82E07C0F601019065
:101BE0000020E9F73197FE2EFC18198240E090C0E2
:101BF00095E5B91621F0A5E7BA1631F402C0B1E0B7
:101C00003B2A7AE0272E16C0E8E5BE1621F0F8E759
:101C1000BF1609F070C033FE0BC02EA53FA548A922
:101C200059A9211531054105510511F030E4332A38
:101C300060E1262E19824AA947FD02C05FED3522D8
:101C40008EA59FA5A8A9B9A90097A105B10549F43A
:101C50009AA9992331F45EE2C52ED12CCC0EDD1E5B
:101C600046C06EA47FA488A899A84EE2C42ED12CA9
:101C7000CC0EDD1EE22CFF2400E010E06EA57FA557
:101C800088A999A9A80197010E946F4B6A3020F496
:101C900030E3A32EA60E08C027E5A22EA60EA8E5C7
:101CA000BA1611F4BFEDAB22F601A2926F016EA538
:101CB0007FA588A999A9A80197010E946F4B2EA71B
:101CC0003FA748AB59AB6E147F048006910618F00D
:101CD00039014A01D3CFF8E02F1649F433FE07C08B
:101CE00020E3A21621F080E3D6018E936D01FCA8BB
:101CF000FC184AA90DC0BB2009F456C0BE82198247
:101D000096E0C92ED12CCC0EDD1E40E0FF24F394CA
:101D1000E42EEF18E7FCEE248981882319F08F2D3B
:101D20008F5F06C036FC02C08F2D02C08F2D8E5FE4
:101D3000A82EAE0C032D10E080E3882E912C80227B
:101D400091228114910421F48BA98A190E94140C08
:101D50008981882329F061E070E0CE01019609C0F5
:101D600006FF09C080E38C83BD8262E070E0CE0193
:101D700004960E94350CB0E28B16910421F48BA9D5
:101D80008A190E94090C8E2D0E94090C6F2D77274D
:101D900067FD7095C6010E94350C04FFABCD8BA981
:101DA0008A190E94140CA6CDE5960FB6F894DEBFF2
:101DB0000FBECDBFDF91CF911F910F91FF90EF909C
:101DC000DF90CF90BF90AF909F908F907F906F905B
:101DD0005F904F903F902F9008951F920F920FB6F3
:101DE0000F9211242F933F935F936F937F938F9361
:101DF0009F93AF93BF938091DF04882329F0809154
:101E0000DF0481508093DF048091E204815080934D
:101E1000E2048F3FB9F489E08093E20480911003DB
:101E20008F5F817080931003882319F481E0809381
:101E3000DA048091D8049091D90401969093D90442
:101E40008093D8048091DD049091DE040297B8F06D
:101E50008091DD049091DE0401979093DE048093DD
:101E6000DD048091DD049091DE0420910B0330911C
:101E70000C0382239323892B09F071C006C08FEFD6
:101E80009FEF90930C0380930B03809100018A30A5
:101E900039F404C05A9A05C0479A03C05A9801C041
:101EA00047988091A40883FF60C0349B0AC080914A
:101EB000DB049091DC0401969093DC048093DB04B6
:101EC00054C08091DB049091DC04892B69F18091EE
:101ED000DB049091DC048A56914030F52091DB04BC
:101EE0003091DC048091DB049091DC0469E270E0C5
:101EF0000E94484B260F371F3093DC042093DB04ED
:101F00008091DB049091DC040B9750F08091DB040E
:101F10009091DC040A97909368058093670504C04C
:101F20001092680510926705809167059091680589
:101F30002091690530916A05845E9D4F821B930B49
:101F400068E671E00E945C4B845B904090936C0566
:101F500080936B051092DC041092DB0406C0809124
:101F600000018A3009F098CF95CFBF91AF919F9132
:101F70008F917F916F915F913F912F910F900FBE45
:101F80000F901F9018952091D8043091D9042F5F9D
:101F90003F4F820F931F08952091D8043091D904A8
:101FA000821B930B892F99278695807490E0089562
:101FB0001F920F920FB60F9211248F939F938091CF
:101FC000090390910A03892B11F05F9A01C05F9871
:101FD00083E08093B000809170008E7F80937000CA
:101FE0009F918F910F900FBE0F901F9018951F9289
:101FF0000F920FB60F921124EF92FF920F931F933F
:102000002F933F934F935F936F937F938F939F9300
:10201000AF93BF93CF93DF93EF93FF938091090327
:1020200090910A03049709F0ACC02091AA0330E014
:10203000220F331F40910D0350910E03CA01880FE8
:10204000991F840F951F280F391F359527953595B2
:10205000279530930E0320930D03205D3F4F30935F
:10206000E1042093E0048091BF0843E0849FC00115
:1020700011242817390740F08091C008849FC001BF
:1020800011248217930720F49093E1048093E004D5
:102090008091CF0820912B0530912C0540912D0582
:1020A00050912E0580FF0FC080913305909134052B
:1020B000A0913505B091360579018A01E81AF90A2F
:1020C0000A0B1B0B02C079018A018091E208209162
:1020D000BE08C091E004D091E10480FF17C030E059
:1020E00040E050E0C801B7010E941D4B57E09595B4
:1020F0008795779567955A95D1F720E830E040E0CD
:1021000050E00E94914BC20FD31F16C030E040E058
:1021100050E0C801B7010E941D4B47E09595879597
:10212000779567954A95D1F720E830E040E050E098
:102130000E94914BC21BD30BD093E104C093E004E7
:102140002091E0043091E10430933B0820933A0859
:10215000C9016FEF70E00E94484B8D9740F4235BFC
:102160003F4F3093E1042093E00483E101C080E617
:1021700080930F038091E00480958093B30083ECFB
:1021800040C08091090390910A03892B39F1809115
:10219000090390910A03049708F52091E004309117
:1021A000E1042F3F310561F058F05F9A83E080939E
:1021B000B0002F5F30403093E1042093E00423C04F
:1021C00083E88093B00080910F038093B30081E097
:1021D00090E090930A038093090315C0809109034E
:1021E00090910A03892B79F48091C10890E0880FBF
:1021F000991F880F991F90930A03809309035F9892
:1022000083E08093B0008091090390910A030197C5
:1022100090930A0380930903FF91EF91DF91CF918F
:10222000BF91AF919F918F917F916F915F914F91EE
:102230003F912F911F910F91FF90EF900F900FBE44
:102240000F901F9018958091D8049091D9040B9607
:102250009093E4048093E30482E085BD83EA84BD27
:1022600017BC88E788BD86E086BD83EC8093B0000C
:1022700084E08093B100E0E7F0E0808182608083B9
:10228000EEE6F0E08081816080838AE08093B30095
:102290001092B2000895AC012091D8043091D90475
:1022A0002F5F3F4F03C08FEE80937A008091D80458
:1022B0009091D904B901681B790BCB01840F951F4C
:1022C00080709078892F99278695882361F30895E7
:1022D000AC012091D8043091D9042F5F3F4F8091F9
:1022E000D8049091D904B901681B790BCB01840FF4
:1022F000951F80709078892F99278695882379F388
:10230000089510927C008FEE80937A0008951F92BA
:102310000F920FB60F921124EF92FF920F931F931B
:102320002F933F934F935F936F937F938F939F93DD
:10233000AF93BF93EF93FF9310927A0080910705BC
:102340008F5F809307058150853009F486C0863001
:1023500090F4823009F440C0833030F48823F1F0E7
:10236000813009F05CC22FC0833009F441C0843051
:1023700009F055C25AC0883009F4D5C0893038F404
:10238000863009F483C0873009F049C2AFC0893074
:1023900009F4E6C08A3009F042C2D9C180917800C0
:1023A00090917900909306058093050581E08093D4
:1023B00008058091FA049091FB0401969093FB0428
:1023C0008093FA0430C280917800909179009093C4
:1023D000040580930305A5C0809178009091790051
:1023E000909302058093010584E0809308051BC249
:1023F00040911103509112038091780090917900DF
:102400009A01220F331F240F351F63E070E00E94F2
:10241000484B260F371F36952795369527953093CD
:1024200012032093110386E0E0CF209178003091D1
:1024300079008091210590912205821B930B909346
:1024400055088093540880915408909155089093B2
:10245000EC048093EB0487E0C8CF809178009091E2
:10246000790020911F0530912005821B930B9093DA
:10247000600880935F0880915F0890916008909356
:10248000EE048093ED0410920805CDC18091000107
:102490008A3069F480917800909179002091050547
:1024A00030910605820F931F9695879519C040912C
:1024B000050550910605843169F42091780030912A
:1024C000790088279927841B950B821B930B8150D9
:1024D0009C4F06C08091780090917900840F951FE1
:1024E0009093EA048093E90481E07FCF809100011A
:1024F00020910305309104058A3049F480917800D9
:1025000090917900820F931F9695879506C08091D0
:10251000780090917900820F931F9093E804809344
:10252000E70482E062CF80910001209101053091A3
:1025300002058A3049F48091780090917900820FE9
:10254000931F9695879506C08091780090917900A9
:10255000820F931F9093E6048093E50485E045CFB6
:102560006091780070917900E0902505F090260543
:102570000091270510912805882777FD8095982FD1
:102580000E94024AA80197010E9402490E94CF4975
:102590007093F0046093EF048091EF049091F00445
:1025A00002970CF43EC0609125057091260580913C
:1025B00027059091280520E030E84BE354E40E9481
:1025C0003D4A88230CF078C060912505709126055E
:1025D00080912705909128052AE037ED43EA5CE3D6
:1025E0000E94034960932505709326058093270573
:1025F000909328058091A6059091A705845F91404E
:1026000008F05AC060912505709126058091270534
:10261000909128052DEC3CEC4CEC5DE30E940349C5
:1026200043C08091EF049091F0048F5F9F4F0CF0B6
:1026300043C06091250570912605809127059091F2
:10264000280520E030E849E054E40E94414A181689
:102650009CF5609125057091260580912705909144
:1026600028052AE037ED43EA5CE30E9402496093C3
:102670002505709326058093270590932805809162
:10268000A6059091A705845F9140B0F4609125055F
:102690007091260580912705909128052DEC3CEC42
:1026A0004CEC5DE30E94024960932505709326057A
:1026B000809327059093280581E08093F60480910C
:1026C0007800909179009093570880935608209154
:1026D00063053091640540916505509166058091D0
:1026E000EF049091F004AA2797FDA095BA2F820FCE
:1026F000931FA41FB51F8093630590936405A09357
:102700006505B0936605E0906305F090640500915F
:10271000650510916605609163057091640580916F
:1027200065059091660520E034E040E050E00E94AD
:10273000914BE21AF30A040B150BE0926305F09239
:102740006405009365051093660583E04ECE809185
:102750006408909165082091780030917900820F8B
:10276000931F909365088093640880915C088F5F45
:1027700080935C0880915C08853008F450C080919B
:10278000780090917900909318038093170310922A
:102790005C082091640830916508E0901303F09084
:1027A00014030091150310911603C801B701660FB9
:1027B000771F881F991F6E0D7F1D801F911F442753
:1027C00037FD4095542F620F731F841F951F24E01F
:1027D00030E040E050E00E94914B2093130330938F
:1027E0001403409315035093160320915808309119
:1027F00059088091130390911403A0911503B0918F
:102800001603281B390B309300052093FF04109208
:1028100065081092640830931D0820931C081092DC
:102820000805109207058091080580937C0080912F
:102830000705882319F08FEE80937A00FF91EF91BE
:10284000BF91AF919F918F917F916F915F914F91C8
:102850003F912F911F910F91FF90EF900F900FBE1E
:102860000F901F9018950F931F931092FC041092D5
:10287000FD041092FE040CE810E0133019F40B3044
:1028800008F009E08091E5049091E6048C5F9340A4
:1028900024F48091190381500CC08091E50490913B
:1028A000E6048750944014F411E006C080911903A7
:1028B0008F5F8093190310E08091E7049091E80402
:1028C0008C5F934024F480911A0381500AC0809158
:1028D000E7049091E8048750944034F080911A0303
:1028E0008F5F80931A0301C01F5F8091E90490916C
:1028F000EA048C5F934024F480911B0381500AC04A
:102900008091E9049091EA048750944034F08091DA
:102910001B038F5F80931B0301C01F5F88E08093C0
:102920000E050E94721A809119038A3030F481E0FA
:102930008093FC048AE08093190380911903863FF9
:1029400030F081E08093FC0485EF8093190380913F
:102950001A038A3030F481E08093FD048AE080938A
:102960001A0380911A03863F30F081E08093FD04C2
:1029700085EF80931A0380911B038A3030F481E045
:102980008093FE048AE080931B0380911B03863FA3
:1029900030F081E08093FE0485EF80931B038091EB
:1029A0000E058823E1F710925C088FEE80937A0081
:1029B00080915C088823E1F30A3020F48AE090E0FB
:1029C0000E944B11015009F058CF86E490E00E941C
:1029D0004B111F910F9108950F931F93CF93DF9386
:1029E000A3E0B0E00E94E34B802DC82FD0E0C531BA
:1029F000D10508F02A97C7BD1092F70484E690E04D
:102A00000E944B11809117039091180382559340B7
:102A1000C8F4C0E0D0E016C0C7BD82E390E00E94D9
:102A20004B111F930F931F920E94490C8091170323
:102A3000909118030F900F900F908255934038F0AB
:102A4000219602C008EF11E0CA3FD10528F3A3E0A8
:102A5000B0E00C2E0E94EB4BC09361088CE291E039
:102A60000E944B11DF91CF911F910F910895E6E2E3
:102A7000F3E080E2819383E0E637F807D1F7089529
:102A80001F934091760380910C05481710F44093F2
:102A90000C0580910D05282F30E0C90181709070E0
:102AA000582F882351F080910C05882321F0815004
:102AB00080930C0502C040930C05B90162707070E0
:102AC00021FF0AC080910C05841719F410920C059F
:102AD00003C08F5F80930C05552321F0672B11F005
:102AE00010920C05E6E2F3E080E2819343E0E637E2
:102AF000F407D1F780910C05282F30E08A3040F49C
:102B000081E180930B053F932F9384E195E007C00B
:102B100080E180930B053F932F938FE095E09F9387
:102B20008F9381E08F930E94490C0F900F900F902C
:102B30000F900F9010910C05153009F405C2163056
:102B400090F4123009F4C3C0133030F4112309F1AA
:102B5000113009F0B8C467C0133009F414C114303F
:102B600009F0B1C46CC1183009F496C3193038F4B7
:102B7000163009F416C3173009F0A5C469C31A301A
:102B800009F40DC41A3008F4C6C31B3009F09BC405
:102B900048C410920B058FEF94E09F938F9311E040
:102BA0001F930E94490C84E180930B052091000142
:102BB000822F6AE00E943C4B492F50E0822F0E94F6
:102BC0003C4B90E022E630E03F932F932AE030E048
:102BD0003F932F9321E030E03F932F935F934F93E8
:102BE0009F938F938AEE94E09F938F931F930E94FD
:102BF000490C88E280930B050E94B80290E09F93F5
:102C00008F938DED94E09F938F931F930E94490CB7
:102C10008CE380930B058DEC94E09F938F931F932F
:102C20000E94490C4CC48091A40880FF33C01092CC
:102C30000B0580910706909108069F938F938EEB6A
:102C400094E09F938F931F930E94490C84E180939B
:102C50000B058091FF04909100059F938F938FEA5D
:102C600094E09F938F931F930E94490C88E2809376
:102C70000B058091610890E09F938F9380EA94E028
:102C80009F938F931F930E94490C4DB75EB7415F8E
:102C90005F4F73C084E180930B0589E994E09F93B3
:102CA0008F931F930E94490C88E280930B058BE859
:102CB00094E09F938F931F930E94490C8DB79EB70A
:102CC00006960FB6F8949EBF0FBE8DBF01C410923A
:102CD0000B0581E894E09F938F9311E01F930E946E
:102CE000490C84E180930B0560912B0570912C05B4
:102CF00080912D0590912E0520E034E040E050E0D9
:102D00000E94914B5F934F933F932F9382E794E000
:102D10009F938F931F930E94490C88E280930B0529
:102D20006091330570913405809135059091360599
:102D300020E034E040E050E00E94914B5F934F93DD
:102D40003F932F9383E694E09F938F931F930E946A
:102D5000490C8CE380930B05809167059091680581
:102D60009F938F9384E594E09F938F931F930E948A
:102D7000490C4DB75EB74A5E5F4F0FB6F8945EBF21
:102D80000FBE4DBFA5C310920B05809172089091A4
:102D9000730820917008309171089F938F933F932F
:102DA0002F9384E494E09F938F9311E01F930E94EC
:102DB000490C84E180930B05809176089091770807
:102DC00020917408309175089F938F933F932F93B0
:102DD00084E394E09F938F931F930E94490C88E2B1
:102DE00080930B0580917A0890917B082091780858
:102DF000309179089F938F933F932F9384E294E0CF
:102E00009F938F931F930E94490C8CE380930B0533
:102E100080917E0890917F0820917C0830917D08F8
:102E20009F938F933F932F9384E194E09F938F938D
:102E30001F930E94490C8DB79EB74C9642CF1092BB
:102E40000B05E0919D08F0E0EE0FFF1FE259F74FF0
:102E500020813181E0919C08F0E0EE0FFF1FE259E4
:102E6000F74F808191813F932F939F938F9384E0BD
:102E700094E09F938F9311E01F930E94490C84E18B
:102E800080930B05E0919F08F0E0EE0FFF1FE259E1
:102E9000F74F20813181E0919E08F0E0EE0FFF1F97
:102EA000E259F74F808191813F932F939F938F93A6
:102EB00084EF93E09F938F931F930E94490C88E2C5
:102EC00080930B05E091A108F0E0EE0FFF1FE2599F
:102ED000F74F20813181E091A008F0E0EE0FFF1F55
:102EE000E259F74F808191813F932F939F938F9366
:102EF00084EE93E09F938F931F930E94490C8CE381
:102F000080930B05E091A308F0E0EE0FFF1FE2595C
:102F1000F74F20813181E091A208F0E0EE0FFF1F12
:102F2000E259F74F808191813F932F939F938F9325
:102F300084ED93E09F938F931F930E94490C4DB7AC
:102F40005EB7445E5F4F19CF10920B0586EC93E09D
:102F50009F938F9311E01F930E94490C8091000171
:102F60000F900F900F908A3009F04DC084E180934C
:102F70000B0520911505309116058091E50490917F
:102F8000E604821B930B3F932F939F938F9387EBC2
:102F900093E09F938F931F930E94490C88E2809344
:102FA0000B0520911705309118058091E704909149
:102FB000E804821B930B3F932F939F938F9388EA90
:102FC00093E09F938F931F930E94490C8CE380930F
:102FD0000B052091190530911A058091E904909113
:102FE000EA04A901481B590B3F932F935F934F931A
:102FF00089E993E09F938F931F930E94490C8DB7AB
:103000009EB745965ECE8B3019F0843109F05CC0D6
:1030100084E180930B052091150530911605C901B7
:1030200062E070E00E945C4B8091E5049091E604C0
:10303000821B930B7F936F939F938F938AE893E008
:103040009F938F931F930E94490C88E280930B05F6
:103050002091170530911805C90162E070E00E94C7
:103060005C4B8091E7049091E804821B930B7F9363
:103070006F939F938F938BE793E09F938F931F930F
:103080000E94490C8CE380930B0520911905309127
:103090001A05C90162E070E00E945C4B8091E9046E
:1030A0009091EA04281B390B7F936F933F932F93E2
:1030B0008CE693E09F938F931F930E94490C4DB72A
:1030C0005EB74B5E5F4F59CE8D3009F001C284E18F
:1030D00080930B052091190330E0E0911505F091E4
:1030E0001605CF0162E070E00E945C4B8091E50420
:1030F0009091E6048E1B9F0B3F932F937F936F93CA
:103100009F938F9388E593E09F938F931F930E94E3
:10311000490C88E280930B0520911A0330E0E0917E
:103120001705F0911805CF0162E070E00E945C4B3A
:103130008091E7049091E8048E1B9F0B3F932F939F
:103140007F936F939F938F9384E493E09F938F93E8
:103150001F930E94490C8CE380930B05E0911B03A5
:10316000F0E02091190530911A05C90162E070E084
:103170000E945C4B8091E9049091EA04281B390B72
:10318000FF93EF937F936F933F932F9380E393E0AD
:103190009F938F931F930E94490C8DB79EB74B96B8
:1031A00090CD10920B0583E293E09F938F9311E0F3
:1031B0001F930E94490C84E180930B0580911F05A9
:1031C000909120052091ED043091EE049F938F9310
:1031D0003F932F9384E193E09F938F931F930E94DB
:1031E000490C88E280930B0580912105909122057E
:1031F0002091EB043091EC049F938F933F932F9396
:1032000085E093E09F938F931F930E94490C8CE37A
:1032100080930B0560912505709126058091270507
:10322000909128050E94CF4920910A0930910B09FD
:103230007F936F933F932F9386EF92E09F938F93AB
:103240001F930E94490C4DB75EB7485E5F4F95CD06
:1032500084E180930B0580911103909112039F9359
:103260008F9387EE92E09F938F9311E01F930E94BC
:10327000490C88E280930B0580917A0590E09F933A
:103280008F9388ED92E09F938F931F930E94490C38
:103290008DB79EB70A9615CD10920B0589EC92E07A
:1032A0009F938F9311E01F930E94490C84E18093B8
:1032B0000B0580916B0590916C059F938F938AEB22
:1032C00092E09F938F931F930E94490C88E2809312
:1032D0000B0580916705909168059F938F938BEA0A
:1032E00092E09F938F931F930E94490C8CE38093ED
:1032F0000B058091690590916A059F938F938CE9E6
:1033000092E09F938F931F930E94490C4DB75EB735
:103310004E5E5F4F32CD10920B05809172059091F9
:1033200073059F938F9380E992E09F938F9311E0B1
:103330001F930E94490C84E180930B0580917405D2
:10334000909175059F938F9384E892E09F938F935C
:103350001F930E94490C88E280930B0580917605AB
:10336000909177059F938F9388E792E09F938F9337
:103370001F930E94490C8CE380930B058091780584
:10338000909179059F938F938CE692E09F938F9312
:103390001F930E94490C8DB79EB7449692CC109211
:1033A0000B0584E692E09F938F9311E01F930E9498
:1033B000490C84E180930B058091AA0390E09F93D0
:1033C0008F9386E592E09F938F931F930E94490C01
:1033D00088E280930B058091E0049091E1049F9333
:1033E0008F9388E492E09F938F931F930E94490CE0
:1033F0008CE380930B052091C00830E08091BF08DA
:1034000090E03F932F939F938F938AE392E09F9353
:103410008F931F930E94490C4DB75EB74C5E5F4F70
:10342000ACCC10920B058AE292E09F938F9311E04F
:103430001F930E94490C84E180930B052091710732
:10344000332727FD309580917007992787FD909548
:103450003F932F939F938F938AE192E09F938F9353
:103460001F930E94490C88E280930B0520917207FC
:10347000332727FD30958091730790E03F932F937A
:103480009F938F938AE092E09F938F931F930E9464
:10349000490C8CE380930B052091770730E08091F5
:1034A0007407992787FD90953F932F939F938F9350
:1034B0008AEF91E09F938F931F930E94490C8DB7E1
:1034C0009EB74896FECB11501093760310920C05D0
:1034D00010920D051F9108951092B9008AE2809311
:1034E000B800089585EA8093BC0080E090E00895DC
:1034F00084E98093BC0008951092B9008093BB00CA
:1035000085E88093BC0080E090E008951F920F92C0
:103510000FB60F9211248F939F93EF93FF93809197
:103520000E058F5F80930E058150E82FF0E0E731A4
:10353000F10508F091C0E85CFF4FEE0FFF1F05900A
:10354000F491E02D099480910F05880F8E5A0CC0DC
:1035500080910F058F5F80930F05815029C08330C4
:1035600009F07AC0809122091092B9008093BB00C3
:1035700085E88093BC0070C084E98093BC00809192
:103580000F05843018F410920E054AC010920F05F2
:1035900047C080911005880F8D5AE6CF8091BB00FF
:1035A000E0911005F0E0EA59F74F80838091100513
:1035B000813041F0813018F0823039F0D0CF8091E5
:1035C000F708D2CF80910009CFCF80911F09CCCFCF
:1035D000809110059091BB00E82FF0E0EA59F74F79
:1035E00094838F5F80931005843058F110921005FA
:1035F00028C01092B90080E1B9CF80911903B4CFEF
:103600001092B90082E1B2CF80911A03ADCF84E964
:103610008093BC008AE090E09093920380939103A2
:1036200085EAA7CF1092B90088E9A0CF1092B9001F
:1036300084E19CCF80911B0397CF1092B90080E862
:1036400095CF84E98093BC008AE090E09093920348
:103650008093910310920E058091BC008068809346
:10366000BC00FF91EF919F918F910F900FBE0F9033
:103670001F9018954CEB50E084E9DA018C9310927E
:103680000E052BEB30E0F901808110920F0580E8E8
:103690008C931092BD001092BA001082E9EBF0E01A
:1036A0001082A8EBB0E01C9210828AE28C9385EA2B
:1036B000DA018C931082F901108285E88C930895C9
:1036C00083EC80938100EFE6F0E08081806280836C
:1036D00010921A05109219051092180510921705EC
:1036E000109216051092150508951F920F920FB6AD
:1036F0000F9211240F931F932F933F934F935F9338
:103700006F937F938F939F93AF93BF93CF93DF93E9
:10371000EF93FF93209186003091870080911305ED
:1037200090911405281B390B809186009091870099
:103730009093140580931305C9018D549440009112
:10374000110510911205835F9A4160F40430110550
:1037500014F01092770381E090E09093120580932B
:1037600011058AC00A3011050CF086C0C9018B5FB3
:103770009040845B914008F068C0E901C25DD1408F
:10378000F801EE0FFF1FE259F74F808191819E01F2
:10379000281B390BC90137FF03C0909581959F4FB6
:1037A00006974CF480917A05883C28F480917A053C
:1037B000865F80937A05F801EE0FFF1FE259F74FFD
:1037C00020813181C901880F991F820F931F8C0FAF
:1037D0009D1F64E070E00E945C4B9B01CE0101964E
:1037E000861797071CF42150304006C021976C17AC
:1037F0007D0714F42F5F3F4F80917A05E801CC0FCD
:10380000DD1F833CB8F0FE01E259F74F80819181C2
:10381000A901481B590BCA0163E070E00E945C4B90
:10382000CB01880F991F860F971FCC57D74F9983CD
:10383000888304C0CC57D74F19821882F801EE0F45
:10384000FF1FE259F74F31832083F8013196F0933F
:103850001205E0931105E530F10511F45D9A06C0FB
:103860005D98E630F10511F45C9A05C05C983797D5
:1038700011F45B9A01C05B98FF91EF91DF91CF91BA
:10388000BF91AF919F918F917F916F915F914F9178
:103890003F912F911F910F910F900FBE0F901F908E
:1038A000189581E080939C0882E080939D0883E0D6
:1038B00080939E0884E080939F0885E08093A00811
:1038C00086E08093A10887E08093A20888E0809337
:1038D000A30808952F923F924F925F926F927F922A
:1038E0008F929F92AF92BF92CF92DF92EF92FF9210
:1038F0000F931F93CF93DF93CDB7DEB726970FB605
:10390000F894DEBF0FBECDBF2091E9043091EA04E8
:103910008091190590911A05821B930B90932C09A5
:1039200080932B092091E9043091EA0480911909D0
:1039300090911A09821B930B90939B0880939A088D
:103940008091E7049091E8042091170530911805C3
:10395000821B930B9093F6088093F5088091E50401
:103960009091E6042091150530911605821B930B6A
:1039700090930209809301096091ED047091EE0427
:10398000882777FD8095982F2CE030E040E050E0CC
:103990000E941D4B9B01AC01609126097091270983
:1039A000882777FD8095982F620F731F841F951FBE
:1039B00022E030E040E050E00E94914B3093270934
:1039C000209326096091EB047091EC04882777FD21
:1039D0008095982F2CE030E040E050E00E941D4B95
:1039E0009B01AC016091390970913A09882777FDF4
:1039F0008095982F620F731F841F951F22E030E07F
:103A000040E050E00E94914B30933A0920933909ED
:103A10006091EF047091F004882777FD8095982FCE
:103A200020910A0930910B09442737FD4095542F06
:103A3000620F731F841F951F22E030E040E050E0CA
:103A40000E94914B30930B0920930A092091ED04B9
:103A50003091EE04C901880F991F820F931F880FC0
:103A6000991F880F991FAA2797FDA095BA2F20911B
:103A70003B0530913C0540913D0550913E05280F96
:103A8000391F4A1F5B1F20933B0530933C05409331
:103A90003D0550933E052091EB043091EC04C901A3
:103AA000880F991F820F931F880F991F880F991FE6
:103AB000AA2797FDA095BA2F20913F053091400588
:103AC0004091410550914205280F391F4A1F5B1F45
:103AD00020933F05309340054093410550934205A4
:103AE0002091ED043091EE04809112099091130918
:103AF000820F931F90931309809312092091EB0476
:103B00003091EC0480912E0990912F09820F931F20
:103B100090932F0980932E0980912305909124057D
:103B200001969093240580932305E0905608F09029
:103B30005708A0902505B0902605C0902705D09085
:103B40002805609143057091440580914505909149
:103B500046050E94024A3B014C010027F7FC0095F4
:103B6000102FC801B7010E94024AA60195010E94C8
:103B700002499B01AC01C401B3010E9403490E94A8
:103B8000CF49609343057093440580934505909316
:103B9000460580912B0990912C099C01442737FD03
:103BA0004095542F8091350990913609A09137099D
:103BB000B0913809280F391F4A1F5B1F2093350920
:103BC00030933609409337095093380980912B0977
:103BD00090912C093C01882477FC8094982C80914A
:103BE0005B0590915C05A0915D05B0915E05680E46
:103BF000791E8A1E9B1E60925B0570925C05809206
:103C00005D0590925E05283787E1380787E0480711
:103C100080E0580764F028573741474050402093D0
:103C2000350930933609409337095093380980910C
:103C3000350990913609A0913709B0913809B7FF3D
:103C40000CC08858984EA84FBF4F80933509909369
:103C50003609A0933709B0933809E0918C05EE83BB
:103C6000EE2309F08AC080918D05882309F085C074
:103C70008091A40886FF81C060919A0870919B088A
:103C8000E0909A05FF2400E010E0882777FD8095FA
:103C9000982F20914B0530914C0540914D05509146
:103CA0004E050E941D4B20E038E040E050E00E94AD
:103CB000914BCA01B901A80197010E941D4B20E058
:103CC00030E140E050E00E94914B59016A0120939D
:103CD000EE053093EF054093F0055093F1056091A8
:103CE0009A0870919B08882777FD8095982F2091DE
:103CF00053053091540540915505509156050E9449
:103D00001D4B20E038E040E050E00E94914BCA019A
:103D1000B901A80197010E941D4B20E030E140E06D
:103D200050E00E94914B2093EA053093EB054093BD
:103D3000EC055093ED05D601C501D7FE07C0B0953F
:103D4000A095909581959F4FAF4FBF4F81389105BA
:103D5000A105B10574F457FF07C050954095309503
:103D600021953F4F4F4F5F4F213831054105510598
:103D7000A4F081E080936F0510C01092EA051092C4
:103D8000EB051092EC051092ED051092EE051092E5
:103D9000EF051092F0051092F1058091F5089091D1
:103DA000F6082091EE053091EF054091F005509115
:103DB000F1052A833B834C835D83820F931F90938D
:103DC000F6088093F5080091F5081091F608A09088
:103DD000EA05B090EB05C090EC05D090ED05809120
:103DE0009B05282E332444245524C201B101A60189
:103DF00095010E941D4B20E032E040E050E00E941F
:103E0000914B020F131F1093F6080093F5082091B1
:103E1000F5083091F608442737FD4095542F8091DE
:103E2000570590915805A0915905B0915A05820FF8
:103E3000931FA41FB51F8093570590935805A09317
:103E40005905B0935A058091F5089091F608209194
:103E5000880530918905821B930BAA2797FDA095B1
:103E6000BA2F20915305309154054091550550913A
:103E70005605820F931FA41FB51F8093530590937F
:103E80005405A0935505B0935605E0909903F09022
:103E90009A0300919B0310919C03E816F9060A0708
:103EA0001B07C4F488EA91E6A0E0B0E08E199F09F0
:103EB000A00BB10B8093530590935405A093550527
:103EC000B09356058093570590935805A0935905D4
:103ED000B0935A0522273327A9012E193F09400B19
:103EE000510B8091530590915405A0915505B091C7
:103EF000560582179307A407B507B4F4D801C70184
:103F0000885A9146A040B040809353059093540541
:103F1000A0935505B0935605809357059093580587
:103F2000A0935905B0935A058091E7049091E80455
:103F30000F9734F488E19CEF9093F6088093F5088E
:103F40008091E7049091E804079734F480E398EFB8
:103F50009093F6088093F5083091000139833A3048
:103F6000A9F48091E7049091E804835F934034F0D2
:103F700088EE93E09093F6088093F5088091E7042B
:103F80009091E8048A5F9340DCF014C08091E704CC
:103F90009091E804855E974034F088EE93E090932A
:103FA000F6088093F5088091E7049091E804835F18
:103FB000974034F080ED97E09093F6088093F508F1
:103FC00080910109909102098A199B099093020935
:103FD000809301090091010910910209C201B10108
:103FE0002A813B814C815D810E941D4B20E032E0A3
:103FF00040E050E00E94914B021B130B109302090A
:10400000009301092091010930910209442737FDED
:104010004095542F80914F0590915005A0915105E6
:10402000B0915205820F931FA41FB51F80934F05B7
:1040300090935005A0935105B093520580910109CA
:104040009091020920918A0530918B05821B930B78
:10405000AA2797FDA095BA2F20914B0530914C05CA
:1040600040914D0550914E05820F931FA41FB51F1F
:1040700080934B0590934C05A0934D05B0934E054E
:10408000E0909503F09096030091970310919803A8
:10409000E816F9060A071B07C4F488EA91E6A0E0CF
:1040A000B0E08E199F09A00BB10B80934B05909344
:1040B0004C05A0934D05B0934E0580934F0590930A
:1040C0005005A0935105B093520522273327A9012B
:1040D0002E193F09400B510B80914B0590914C05D7
:1040E000A0914D05B0914E0582179307A407B5071F
:1040F000B4F4D801C701885A9146A040B0408093DB
:104100004B0590934C05A0934D05B0934E058093BD
:104110004F0590935005A0935105B093520580919F
:10412000E5049091E6040F9734F488E19CEF9093B6
:104130000209809301098091E5049091E6040797B4
:1041400034F480E398EF9093020980930109298168
:104150002A30A9F48091E5049091E604835F9340AE
:1041600034F088EE93E090930209809301098091E6
:10417000E5049091E6048A5F9340DCF014C08091DE
:10418000E5049091E604855E974034F088EE93E074
:1041900090930209809301098091E5049091E604CF
:1041A000835F974034F080ED97E09093020980930D
:1041B00001098FEE80937A0060924705709248055E
:1041C0008092490590924A0580914B0590914C054B
:1041D000A0914D05B0914E0580932B0590932C0531
:1041E000A0932D05B0932E05809153059091540511
:1041F000A0915505B09156058093330590933405F1
:10420000A0933505B093360580914F0590915005E8
:10421000A0915105B091520580932F0590933005E0
:10422000A0933105B09332058091570590915805C0
:10423000A0915905B0915A058093370590933805A0
:10424000A0933905B0933A058091A40887FF63C015
:10425000FE81FF2309F05FC080918D05882309F05E
:104260005AC08091010990910209893C91055CF046
:104270002091010930910209809101099091020970
:104280002052334011C08091010990910209885356
:104290009F4FA4F4209101093091020980910109F6
:1042A00090910209205E3C4F880F991F880F991F3B
:1042B000280F391F30930209209301098091F508D6
:1042C0009091F608893C91055CF02091F5083091B9
:1042D000F6088091F5089091F6082052334011C0FD
:1042E0008091F5089091F60888539F4FA4F420918F
:1042F000F5083091F6088091F5089091F608205E57
:104300003C4F880F991F880F991F280F391F309332
:10431000F6082093F508209172053091730580917D
:10432000A008E82FF0E0EE0FFF1FE259F74F808161
:10433000918182599F4F281739071CF42F5F3F4FF7
:104340000CC08081918182599F4F821793074CF452
:104350002115310531F02150304030937305209301
:10436000720520917405309175058091A108E82FA0
:10437000F0E0EE0FFF1FE259F74F808191818259E3
:104380009F4F281739071CF42F5F3F4F0CC08081C7
:10439000918182599F4F821793074CF42115310563
:1043A00031F02150304030937505209374052091F1
:1043B0007605309177058091A208E82FF0E0EE0FA6
:1043C000FF1FE259F74F8081918182599F4F281733
:1043D00039071CF42F5F3F4F0CC0808191818259B7
:1043E0009F4F821793074CF42115310531F021506E
:1043F00030403093770520937605209178053091F1
:1044000079058091A308E82FF0E0EE0FFF1FE25935
:10441000F74F8081918182599F4F281739071CF4EB
:104420002F5F3F4F0CC08081918182599F4F82172F
:1044300093074CF42115310531F021503040309371
:10444000790520937805809172059091730597FF07
:1044500005C010927305109272050AC08F3F910536
:1044600039F034F08FEF90E09093730580937205EC
:10447000809174059091750597FF05C010927505A0
:10448000109274050AC08F3F910539F034F08FEF18
:1044900090E09093750580937405809176059091D6
:1044A000770597FF05C010927705109276050AC030
:1044B0008F3F910539F034F08FEF90E090937705BE
:1044C00080937605809178059091790597FF05C0D6
:1044D00010927905109278050AC08F3F910539F046
:1044E00034F08FEF90E090937905809378052696CD
:1044F0000FB6F894DEBF0FBECDBFDF91CF911F91F5
:104500000F91FF90EF90DF90CF90BF90AF909F9072
:104510008F907F906F905F904F903F902F90089575
:104520008091A7088B3F98F08B3F19F4809172051A
:104530000EC08C3F19F48091740509C08D3F19F4A9
:104540008091760504C08E3F21F480917805809398
:10455000A2038091A6088B3F98F08B3F19F48091BD
:1045600072050EC08C3F19F48091740509C08D3F0F
:1045700019F48091760504C08E3F21F4809178056E
:104580008093A1038091A103882319F41092A103C1
:1045900005C0843618F084E68093A1038091A808B2
:1045A0008B3F98F08B3F19F4809172050EC08C3FC1
:1045B00019F48091740509C08D3F19F48091760536
:1045C00004C08E3F21F4809178058093A3038091ED
:1045D000A303882319F41092A30305C0843618F0AE
:1045E00084E68093A3038091AA088B3F98F08B3FC9
:1045F00019F4809172050EC08C3F19F480917405F6
:1046000009C08D3F19F48091760504C08E3F21F4D6
:10461000809178058093A4038091B1088B3F98F036
:104620008B3F19F4809172050EC08C3F19F4809174
:10463000740509C08D3F19F48091760504C08E3F42
:1046400021F4809178058093A5038091B2088B3F77
:1046500098F08B3F19F4809172050EC08C3F19F4CD
:104660008091740509C08D3F19F48091760504C0CE
:104670008E3F21F4809178058093A6038091A60354
:104680008B3010F48AE002C08F3F11F48093A603B0
:104690008091B3088B3F98F08B3F19F4809172059D
:1046A0000EC08C3F19F48091740509C08D3F19F438
:1046B0008091760504C08E3F21F480917805809327
:1046C000A7038091B8088B3F98F08B3F19F4809135
:1046D00072050EC08C3F19F48091740509C08D3F9E
:1046E00019F48091760504C08E3F21F480917805FD
:1046F0008093A9038091B9088B3F98F08B3F19F400
:10470000809172050EC08C3F19F48091740509C028
:104710008D3F19F48091760504C08E3F21F480917D
:104720007805809392058091BA088B3F98F08B3F73
:1047300019F4809172050EC08C3F19F480917405B4
:1047400009C08D3F19F48091760504C08E3F21F495
:1047500080917805809393058091BB088B3F98F0FA
:104760008B3F19F4809172050EC08C3F19F4809133
:10477000740509C08D3F19F48091760504C08E3F01
:1047800021F480917805809394058091BC088B3F3B
:1047900098F08B3F19F4809172050EC08C3F19F48C
:1047A0008091740509C08D3F19F48091760504C08D
:1047B0008E3F21F480917805809395058091CC08F7
:1047C0008B3F98F08B3F19F4809172050EC08C3F9F
:1047D00019F48091740509C08D3F19F48091760514
:1047E00004C08E3F21F480917805809396058091D6
:1047F000CD088B3F98F08B3F19F4809172050EC065
:104800008C3F19F48091740509C08D3F19F4809193
:10481000760504C08E3F21F480917805809397053A
:104820008091CE088B3F98F08B3F19F480917205F0
:104830000EC08C3F19F48091740509C08D3F19F4A6
:104840008091760504C08E3F21F480917805809395
:1048500098058091CF088B3F98F08B3F19F4809199
:1048600072050EC08C3F19F48091740509C08D3F0C
:1048700019F48091760504C08E3F21F4809178056B
:10488000809399058091BD088B3F98F08B3F19F478
:10489000809172050EC08C3F19F48091740509C097
:1048A0008D3F19F48091760504C08E3F21F48091EC
:1048B00078058093AA038091C2088B3F98F08B3FC4
:1048C00019F4809172050EC08C3F19F48091740523
:1048D00009C08D3F19F48091760504C08E3F21F404
:1048E000809178058093AB038091C5088B3F98F049
:1048F0008B3F19F4809172050EC08C3F19F48091A2
:10490000740509C08D3F19F48091760504C08E3F6F
:1049100021F48091780580939A058091C6088B3F99
:1049200098F08B3F19F4809172050EC08C3F19F4FA
:104930008091740509C08D3F19F48091760504C0FB
:104940008E3F21F48091780580939B058091CB0860
:104950008B3F98F08B3F19F4809172050EC08C3F0D
:1049600019F48091740509C08D3F19F48091760582
:1049700004C08E3F21F4809178058093AC03809130
:10498000D1088B3F98F08B3F19F4809172050EC0CF
:104990008C3F19F48091740509C08D3F19F4809102
:1049A000760504C08E3F21F4809178058093140928
:1049B00080911409823010F481E002C08F3F11F41D
:1049C000809314098091D3088B3F98F08B3F19F4A2
:1049D000809172050EC08C3F19F48091740509C056
:1049E0008D3F19F48091760504C08E3F21F48091AB
:1049F00078058093290980912909823010F481E09B
:104A000002C08F3F11F4809329098091E0088B3F09
:104A100098F08B3F19F4809172050EC08C3F19F409
:104A20008091740509C08D3F19F48091760504C00A
:104A30008E3F21F48091780580933C096091A90311
:104A400070E080E090E00E94554727E137EB41EDB0
:104A500058E30E94BA4A60939D0370939E0380932B
:104A60009F039093A0038091AF0880932A098091BF
:104A7000AE088093040908958091F70890E0909320
:104A80002B0880932A088091000990E090932D08CC
:104A900080932C088091220990E090932F088093B6
:104AA0002E0880911F0990E0909331088093300880
:104AB00080918305882321F08091CE0880FD24C059
:104AC000109200091092F70810921F091092220903
:104AD0008091CC04882311F08093F7088091CD0455
:104AE000882311F0809300098091CE04882311F06F
:104AF000809322098091CF04882311F080931F09AD
:104B00008091A8058C7F03C08091A8058160809367
:104B1000A80510920E0510920F050E94721A0895B2
:104B2000809100018D3011F40E94331410927A00AC
:104B30008091E5049091E604909302098093010925
:104B40008091E7049091E8049093F6088093F5082B
:104B50008091E9049091EA0490932C0980932B09A9
:104B60006091ED047091EE04882777FD8095982F71
:104B70002CE030E040E050E00E941D4B709327098C
:104B8000609326096091EB047091EC04882777FD0F
:104B90008095982F0E941D4B70933A0960933909B4
:104BA0008091EF049091F00490930B0980930A098F
:104BB0008FEE80937A002091720530917305809179
:104BC000A008E82FF0E0EE0FFF1FE259F74F8081B9
:104BD000918182599F4F281739071CF42F5F3F4F4F
:104BE0000CC08081918182599F4F821793074CF4AA
:104BF0002115310531F02150304030937305209359
:104C0000720520917405309175058091A108E82FF7
:104C1000F0E0EE0FFF1FE259F74F8081918182593A
:104C20009F4F281739071CF42F5F3F4F0CC080811E
:104C3000918182599F4F821793074CF421153105BA
:104C400031F0215030403093750520937405209148
:104C50007605309177058091A208E82FF0E0EE0FFD
:104C6000FF1FE259F74F8081918182599F4F28178A
:104C700039071CF42F5F3F4F0CC08081918182590E
:104C80009F4F821793074CF42115310531F02150C5
:104C90003040309377052093760520917805309148
:104CA00079058091A308E82FF0E0EE0FFF1FE2598D
:104CB000F74F8081918182599F4F281739071CF443
:104CC0002F5F3F4F0CC08081918182599F4F821787
:104CD00093074CF42115310531F0215030403093C9
:104CE000790520937805809172059091730597FF5F
:104CF00005C010927305109272050AC08F3F91058E
:104D000039F034F08FEF90E0909373058093720543
:104D1000809174059091750597FF05C010927505F7
:104D2000109274050AC08F3F910539F034F08FEF6F
:104D300090E090937505809374058091760590912D
:104D4000770597FF05C010927705109276050AC087
:104D50008F3F910539F034F08FEF90E09093770515
:104D600080937605809178059091790597FF05C02D
:104D700010927905109278050AC08F3F910539F09D
:104D800034F08FEF90E090937905809378056091EF
:104D9000C70870E080E090E024EC39E040E050E0AB
:104DA0000E941D4B60939503709396038093970325
:104DB000909398036091C80870E080E090E00E94B2
:104DC0001D4B6093990370939A0380939B03909378
:104DD0009C0308951092200510921F051092220541
:104DE0001092210580E090E0A0E0B0E080932505DE
:104DF00090932605A0932705B093280510921605D9
:104E000010921505109218051092170510921A05A8
:104E10001092190510921A091092190910929A0508
:104E200010929B051092F7040E94902584E690E072
:104E30000E944B110E9490258091A40880FF10C011
:104E40008091170390911803875B934038F4809109
:104E50001703909118038E5E924010F40E94EC1498
:104E60004091E5045091E6045093160540931505D2
:104E70002091E7043091E80430931805209317053A
:104E80008091E9049091EA0490931A0580931905A2
:104E90008091E9049091EA0490931A09809319098A
:104EA00030931C0520931B0550931E0540931D0550
:104EB00044E050E0DA010E94E34B802D853038F168
:104EC0008091390990913A0997FF03C09095819597
:104ED0009F4F6CE070E00E945C4B709322056093E2
:104EE0002105809126099091270997FF03C090958D
:104EF00081959F4F6CE070E00E945C4B70932005A1
:104F000060931F05609156087091570839C0DA0107
:104F10000E94E34B802D4F5F5F4FDA010E94E34B0D
:104F2000202D90E0982F8827820F911D90932005C7
:104F300080931F054F5F5F4FDA010E94E34B802D86
:104F40004F5F5F4FDA010E94E34B202D90E0982FD6
:104F50008827820F911D90932205809321054F5F32
:104F60005F4FDA010E94E34B602D4F5F5F4FDA0124
:104F70000E94E34B202D70E0762F6627620F711D93
:104F8000882777FD8095982F0E94024A6093250517
:104F900070932605809327059093280510924B0562
:104FA00010924C0510924D0510924E0510924F052F
:104FB000109250051092510510925205109253050F
:104FC00010925405109255051092560510925705EF
:104FD000109258051092590510925A0510925B05CF
:104FE00010925C0510925D0510925E051092020908
:104FF000109201091092F6081092F50810922C09EF
:1050000010922B0984E690E00E944B1180911303CB
:1050100090911403A0911503B09116039093590831
:10502000809358081092F9041092F80410926305C6
:1050300010926405109265051092660580916705CF
:105040009091680590936A05809369050E942B47AB
:1050500082E390E09093DE048093DD046091C708C2
:1050600070E080E090E024EC39E040E050E00E9405
:105070001D4B6856754C8F4F9F4F609395037093EF
:10508000960380939703909398036091C80870E00B
:1050900080E090E00E941D4B6856754C8F4F9F4FEB
:1050A0006093990370939A0380939B0390939C035E
:1050B0001092AE031092AD03609167057091680580
:1050C000882777FD8095982F2BE035E040E050E071
:1050D0000E941D4B60933509709336098093370900
:1050E00090933809109271051092700581E08093B9
:1050F00001010E942B438091A80584608093A8053C
:105100008FEF8093A2098091CA0890E064E0880F35
:10511000991F6A95E1F78093A30980E28093A4091F
:1051200008951F93182F0EC080918305882361F482
:1051300084E690E09093DE048093DD048AEF90E0B3
:105140000E946811115080F71F91089588EE809396
:10515000A4083EE13093A50880E58093A7088AE083
:105160008093A8083093A6083093AA088093A908D2
:1051700058E05093AB0890E19093AC0866E06093E0
:10518000AD085093AE0886EE8093AF083093B00818
:1051900080E88093B10844E64093B20888E78093A2
:1051A000B3088EE58093B40883E28093B50884E168
:1051B0008093B6081092B7089093B80887E0809360
:1051C000B90882E08093BA081092BB081092BC081C
:1051D0001092CC081092CD081092CE081092CF08F1
:1051E0004093BD0888E28093BE081092E20892E3E3
:1051F0009093BF0886E98093C00885E08093C1083A
:105200009093C2082AE52093C3089093C408109293
:10521000E1082093C5088093C60885E58093C708F8
:105220008093C80880E28093C90884E08093CA080C
:105230009093CB088FE58093D00883EF8093D208BA
:105240003093D1083093D3088DEF8093D4084093E6
:10525000D5082093D6082093D7082093D808109219
:10526000D9086093DA085093DB082093DC08309368
:10527000DD084093DE088CE38093DF08A7EEB8E0FA
:10528000E8E7F3E08CE001900D928150E1F708959A
:1052900088E68093A4084EE14093A50890E590939A
:1052A000A7088AE08093A8084093A6084093AA081C
:1052B0008093A9088CE08093AB0880E18093AC08D0
:1052C00076E07093AD0868E06093AE0886EE809358
:1052D000AF084093B00880E88093B1089093B2087B
:1052E00088E78093B3088EE58093B40883E28093C7
:1052F000B5084093B6081092B70850E25093B8082A
:1053000087E08093B90882E08093BA081092BB08C6
:105310001092BC081092CC081092CD081092CE08C2
:105320001092CF0834E63093BD0888E28093BE081F
:105330001092E20892E39093BF0886E98093C00838
:1053400085E08093C1089093C2082AE52093C308A2
:105350009093C4081092E1082093C5088093C60872
:1053600085E58093C7088093C8085093C90884E0F6
:105370008093CA088BE48093CB088FE58093D00894
:1053800083EF8093D20884E18093D1088093D3087F
:105390008DEF8093D4083093D5082093D6082093BE
:1053A000D7082093D8081092D9087093DA08609330
:1053B000DB082093DC084093DD083093DE088CE3A3
:1053C0008093DF08A7EEB8E0E2E8F3E08CE001901C
:1053D0000D928150E1F7089588E68093A4083EE19C
:1053E0003093A50890E59093A7088AE08093A808D9
:1053F0003093A6083093AA088093A9085FE05093E1
:10540000AB083093AC088CE08093AD0868E0609303
:10541000AE0886EE8093AF083093B00880E88093A2
:10542000B1089093B20896E99093B3088EE5809303
:10543000B40883E28093B5083093B6081092B70899
:1054400080E28093B80887E08093B90882E0809377
:10545000BA081092BB081092BC081092CC081092A7
:10546000CD081092CE081092CF0844E64093BD08B4
:1054700088E28093BE081092E20882E38093BF081E
:105480009093C00825E02093C1088093C2089AE554
:105490009093C3088093C4081092E1089093C508C4
:1054A0002093C60885E58093C7088093C80880E1EB
:1054B0008093C90884E08093CA084093CB088FE5A5
:1054C0008093D00883EF8093D2085093D1085093F3
:1054D000D3088DEF8093D4084093D5089093D608D5
:1054E0009093D7089093D8081092D90886E08093BB
:1054F000DA086093DB089093DC083093DD08409372
:10550000DE088CE38093DF08A7EEB8E0EAE8F3E07A
:105510008CE001900D928150E1F708952F923F9217
:105520004F925F926F927F928F929F92AF92BF92B3
:10553000CF92DF92EF92FF920F931F93CF93DF935F
:10554000CDB7DEB7A5970FB6F894DEBF0FBECDBFBF
:105550000E946A1C309100013C3010F4299A01C06D
:10556000299840918105509182055D874C878091F3
:105570007A05843608F06CC080910501882399F47F
:1055800080910B0390910C038F5F9F4F61F488E92A
:105590009AE39093DE048093DD0480E09CE0909396
:1055A0000C0380930B038091CC059091CD0500975F
:1055B00031F001979093CD058093CC0504C01092F3
:1055C000830510926D053A3011F0343111F4289AA8
:1055D00001C028988091A6059091A705895E934007
:1055E000A0F18091B508A82FB0E0BD87AC8781E01D
:1055F00080936D05A0919C08B0E0AA0FBB1FFD0130
:10560000EC57F74F11821082E0919D082E2F30E069
:10561000220F331FC9018C57974FFC011182108252
:10562000A259B74F11961C921E922259374FD90199
:1056300011961C921E92E0919F08F0E0EE0FFF1F62
:10564000E259F74F11821082BBC210928305B8C293
:1056500080917A058D3808F4B3C210926D0580915F
:10566000B60822E3829FC00111249093CD05809358
:10567000CC05EC85FD85B9978CF080918305882356
:1056800069F08091A6059091A705FFEF8F3F9F07D6
:1056900029F001969093A7058093A6058091A60511
:1056A0009091A7058F3F910509F038F51092E60516
:1056B0001092E7051092E8051092E9051092E205B4
:1056C0001092E3051092E4051092E5058A3F9105DA
:1056D000C9F481E08093C7051092DE051092DF05C2
:1056E0001092E0051092E10510925B0510925C05A6
:1056F00010925D0510925E0505C08091A80582603C
:105700008093A805E0919E08F0E0EE0FFF1FE2599C
:10571000F74F80819181813591050CF485C180918D
:105720008305882309F080C180919F08E82FF0E06D
:10573000EE0FFF1FE259F74F808191818C34910564
:105740000CF4E5C08091CB058F5F8093CB05893C3D
:1057500008F46AC13C3010F4299801C0299A1092CB
:1057600083051092CB051092A7051092A605809193
:105770009C08282F30E0F901EE0FFF1FE259F74F88
:1057800080819181873491059CF4E0919D08F0E03F
:10579000EE0FFF1FE259F74F0190F081E02DF7FF68
:1057A00003C0F095E195FF4FE734F1050CF46AC0B2
:1057B00080919D08682F70E0DB01AA0FBB1FA259E2
:1057C000B74F8D919C911197873491053CF0F90169
:1057D000EE0FFF1FE259F74F808191818D919C91CF
:1057E0008734910564F0F901EE0FFF1FE259F74F7E
:1057F000808191818734910514F042E001C041E03D
:10580000FB01EE0FFF1FE259F74F80819181863433
:1058100091055CF4F901EE0FFF1FE259F74F80810B
:105820009181873491050CF043E0FB01EE0FFF1FDF
:10583000E259F74F808191818A5B9F4F5CF4F901B7
:10584000EE0FFF1FE259F74F808191818734910558
:105850000CF044E0660F771F6259774FDB018D91A2
:105860009C918A5B9F4F5CF4220F331F2259374F64
:10587000F90180819181863491050CF445E0842FF3
:105880000E94AC02E0919D08F0E0EE0FFF1FE2598C
:10589000F74F0190F081E02DF7FF03C0F095E195FF
:1058A000FF4F7E97B4F4E0919C08F0E0EE0FFF1FED
:1058B000E259F74F808191818A5B9F4F54F481E0D8
:1058C00080936B0788EE93E09093DE048093DD0471
:1058D000ABC00E94B80246E56CE978E00E941E0366
:1058E0008091A40880FF10C0809117039091180345
:1058F000875B934038F480911703909118038E5E74
:10590000924010F40E94EC140E94EA2686C0808126
:105910009181855B9F4F0CF085C08091CB058F5F97
:105920008093CB05893C08F47FC03C3010F4299863
:1059300001C0299A8FEF04E010E0D801082E0E94E0
:10594000EB4B109283051092CB051092A705109295
:10595000A6050E94EA2680911F059091200560E02F
:1059600071E00E945C4BD801062E0E94EB4B8091A7
:105970001F059091200560E071E00E945C4B0F5F75
:105980001F4FD801082E0E94EB4B8091210590916A
:10599000220560E071E00E945C4B0F5F1F4FD80151
:1059A000062E0E94EB4B809121059091220560E02C
:1059B00071E00E945C4B0F5F1F4FD801082E0E94C0
:1059C000EB4B6091250570912605809127059091FC
:1059D00028050E94CF49DC01CB0160E071E00E9404
:1059E0005C4B0F5F1F4FD801062E0E94EB4B60915E
:1059F00025057091260580912705909128050E9424
:105A0000CF49DC01CB0160E071E00E945C4B0F5F8D
:105A10001F4FD801082E0E94EB4B0E94B8020E9433
:105A2000912802C01092CB05E0919E08F0E0EE0FA5
:105A3000FF1FE259F74F808191818B5A9F4F0CF0E5
:105A4000BFC080918305882309F099C0E0919F0829
:105A5000F0E0EE0FFF1FE259F74F80819181855BE7
:105A60009F4F0CF08CC08091CA058F5F8093CA0550
:105A7000893C08F486C088EC8093CA0581E090E0F8
:105A80009093A7058093A60581E0809383051092EB
:105A9000DE051092DF051092E0051092E1051092EC
:105AA0005B0510925C0510925D0510925E051092E8
:105AB0005F051092600510926105109262051092C8
:105AC0004B0510924C0510924D0510924E05109208
:105AD0005305109254051092550510925605809169
:105AE0002B0590912C05A0912D05B0912E0580934A
:105AF0004F0590935005A0935105B09352058091A6
:105B0000330590913405A0913505B0913605809309
:105B1000570590935805A0935905B0935A051092D4
:105B2000E6051092E7051092E8051092E90510923B
:105B3000E2051092E3051092E4051092E5058091CC
:105B4000A80588608093A8058091CF0881FF19C0BF
:105B50008091A40880FF10C08091170390911803D2
:105B6000875B934038F480911703909118038E5E01
:105B7000924010F40E94EC140E94EA2602C0109297
:105B8000CA05E0919F08F0E0EE0FFF1FE259F74FC2
:105B9000808191818C3491058CF08091C9058F5F53
:105BA0008093C905893C60F01092830588EC80934E
:105BB000C9051092A7051092A60502C01092C9054A
:105BC00080917703815080937703809177038F3F93
:105BD00029F080916D05882309F499C30E949022D1
:105BE000E0919C08F0E0EE0FFF1FE259F74F808133
:105BF00091811C01442437FC4094542CE0919D0871
:105C0000F0E0EE0FFF1FE259F74F808191813C01D8
:105C1000882477FC8094982C8091CF08482F50E0FE
:105C20005DA34CA380FF76C0EE24FF248701E61815
:105C3000F70808091909C201B1012FE93BE140E069
:105C400050E00E941D4B5B016C01C801B7010E942E
:105C50001D4B7B018C01C601B5016E197F09800BBC
:105C6000910B20E137E240E050E00E94914B190196
:105C7000442437FC4094542CEA0CFB1C0C1D1D1DC5
:105C8000C801B70120E137E240E050E00E94914BAB
:105C9000309521953F4F3901882477FC8094982CCA
:105CA0005EE7251631044104510434F04DE7242EFB
:105CB000312C412C512C11C063E826166FEF3606AB
:105CC0006FEF46066FEF560644F433E8232E3FEF9E
:105CD000332E3FEF432E3FEF532E7EE767167104BE
:105CE0008104910434F02DE7622E712C812C912CCB
:105CF00011C083E868168FEF78068FEF88068FEF64
:105D0000980644F493E8692E9FEF792E9FEF892E31
:105D10009FEF992E8091BD059091BE05AA2797FD12
:105D2000A095BA2FA2019101281B390B4A0B5B0BDE
:105D3000CA01B90123E030E040E050E00E94914BFD
:105D400079018A01EE0CFF1C001F111FE20EF31EE9
:105D5000041F151F8091BB059091BC05AA2797FDD4
:105D6000A095BA2FA4019301281B390B4A0B5B0B9A
:105D7000CA01B90123E030E040E050E00E94914BBD
:105D800059016A01AA0CBB1CCC1CDD1CA20EB31E5F
:105D9000C41ED51EC1013092BE052092BD0523014F
:105DA0007092BC056092BB056090AB087724809030
:105DB000AC089924E89CF001E99CF00DF89CF00DEA
:105DC0001124AC01469DC001479D900D569D900D3C
:105DD00011244091B9055091BA059A01220F331F41
:105DE000240F351F820F931F64E070E00E945C4B0C
:105DF000E60FF71FF093BA05E093B90580911506F9
:105E000090911606E81BF90BF0937C05E0937B0557
:105E1000A89CF001A99CF00DB89CF00D1124469CA3
:105E2000C001479C900D569C900D11244091B705E0
:105E30005091B8059A01220F331F240F351F820F8E
:105E4000931F64E070E00E945C4BE60FF71FF09335
:105E5000B805E093B7058091170690911806E81BE6
:105E6000F90BF0937E05E0937D05E0919F08F0E04B
:105E7000EE0FFF1FE259F74F808191819095819538
:105E80009F4F9093800580937F056CA17DA16072E8
:105E900070707DA36CA38091BA0390E0682B792B7E
:105EA000672B19F00E9409440BC0E0919E08F0E0B6
:105EB000EE0FFF1FE259F74F8081918188589F4F65
:105EC00090938205809381056091A60370E080E045
:105ED00090E00E94554720E030E040E251E40E940B
:105EE000034920E030E040E85CE30E94BA4A7B01CD
:105EF0008C0160933009709331098093320990933B
:105F000033096091A70370E080E090E00E9455475C
:105F100020E030EE4BE256E40E94674960931B0993
:105F200070931C0980931D0990931E098091770737
:105F300080FF67C080913C09813808F462C02091DD
:105F4000AB0830E080917007992787FD9095289FD6
:105F5000A001299F500D389F500D112480917B0581
:105F600090917C05840F951F90937C0580937B0511
:105F700080917107992787FD9095D9018A9F90019B
:105F80008B9F300D9A9F300D112480917D0590914B
:105F90007E05820F931F90937E0580937D0520914F
:105FA0007207332727FD309580917F0590918005FA
:105FB000820F931F9093800580937F052091A908FD
:105FC00030E080917407992787FD9095FC012E9F02
:105FD000C0012F9F900D3E9F900D11249093AE0312
:105FE0008093AD0380917307282F30E08091810565
:105FF000909182052817390724F430938205209365
:106000008105809181059091820597FF04C01092CF
:106010008205109281058091A40882FF0CC080E067
:1060200090E0A0E0B0E080931B0990931C09A0933E
:106030001D09B0931E0920E030E040E050E0C801A7
:10604000B7010E943D4A882364F480E090E0A0E01C
:10605000B0E08093300990933109A0933209B09356
:10606000330920E030E040E050E060911B0970917E
:106070001C0980911D0990911E090E943D4A8823A8
:1060800064F480E090E0A0E0B0E080931B0990937E
:106090001C09A0931D09B0931E09E0917B05F091A6
:1060A0007C052091A2053091A305CF0164E070E04A
:1060B0000E945C4B77FF03C0709561957F4F261758
:1060C0003707C4F4CF01F7FF03C0909581959F4F28
:1060D00064E070E00E945C4B7093A3056093A2059E
:1060E000653671056CF084E690E09093A30580938B
:1060F000A20506C0215030403093A3052093A2058D
:10610000E0917D05F0917E052091A4053091A505D3
:10611000CF0164E070E00E945C4B77FF03C0709594
:1061200061957F4F26173707C4F4CF01F7FF03C0EF
:10613000909581959F4F64E070E00E945C4B709356
:10614000A5056093A405653671056CF084E690E0C2
:106150009093A5058093A40506C02150304030934C
:10616000A5052093A40580916D05882341F0109228
:10617000A3051092A2051092A5051092A405809186
:106180009D08A82FB0E0FD01EE0FFF1FE259F74F69
:10619000208131818091C308482F50E04217530776
:1061A00044F48091E10882FF04C081E080938E0571
:1061B00011C0FD01EE0FFF1FE259F74F2081318121
:1061C0008091C408BA01681B71092617370714F4B7
:1061D00010928E05FD01EE0FFF1FE259F74F8081EF
:1061E000918166277727641B750B8617970744F400
:1061F0008091E10883FF04C081E080938F0514C083
:1062000080918F05882381F0AA0FBB1FA259B74F39
:106210002D913C918091C40890E0841B950B8217CE
:10622000930714F410928F0580919C08A82FB0E07A
:10623000FD01EE0FFF1FE259F74F80819181481752
:10624000590744F48091E10880FF04C081E0809305
:10625000910515C080919105882389F0FD01EE0F0D
:10626000FF1FE259F74F208131818091C408FA0164
:10627000E81BF1092E173F0714F410929105FD0158
:10628000EE0FFF1FE259F74F808191818617970724
:1062900044F48091E10881FF04C081E0809390057F
:1062A00014C080919005882381F0AA0FBB1FA259CA
:1062B000B74F2D913C918091C40890E0841B950BC1
:1062C0008217930714F41092900580918E0588230D
:1062D00021F480918F05882321F081E080938D0542
:1062E00002C010928D0580919105882321F4809140
:1062F0009005882351F081E080938C0510928D05E4
:1063000010928E0510928F0502C010928C0580911C
:106310008D05882321F480918C05882351F080918C
:10632000C20890E02C853D858217930714F49D8761
:106330008C8780916D05882341F110928005109221
:106340007F0510927C0510927B0510927E051092BD
:106350007D0580E090E0A8ECBFE380933009909346
:106360003109A0933209B09333098BE09CEBA2E38F
:10637000BCE380931B0990931C09A0931D09B09363
:106380001E0910928D0510928C0540912B0550919D
:106390002C0560912D0570912E054A835B836C83DB
:1063A0007D8380910E0990910F09A0911009B09101
:1063B0001109840F951FA61FB71F80930E09909394
:1063C0000F09A0931009B0931109609133057091E2
:1063D00034058091350590913605688779878A87DD
:1063E0009B878091150990911609A0911709B0918A
:1063F0001809288539854A855B85820F931FA41F5C
:10640000B51F8093150990931609A0931709B093AF
:10641000180940912F055091300560913105709118
:10642000320548A359A36AA37BA3809106099091E2
:106430000709A0910809B0910909840F951FA61FAB
:10644000B71F8093060990930709A0930809B0939A
:10645000090960913705709138058091390590914F
:106460003A056C8F7D8F8E8F9F8F8091FB08909166
:10647000FC08A091FD08B091FE082C8D3D8D4E8D3D
:106480005F8D820F931FA41FB51F8093FB0890930D
:10649000FC08A093FD08B093FE0830918C05398369
:1064A000332329F480918D05882309F460C010926C
:1064B0003B0510923C0510923D0510923E0510924E
:1064C0003F0510924005109241051092420510922E
:1064D0000E0910920F0910921009109211091092D2
:1064E00015091092160910921709109218091092A6
:1064F00006091092070910920809109209091092D2
:10650000FB081092FC081092FD081092FE08809182
:106510004B0590914C05A0914D05B0914E0580938F
:106520004F0590935005A0935105B093520580916B
:10653000530590915405A0915505B091560580934F
:10654000570590935805A0935905B0935A0510929A
:10655000FB041092FA0410928B0510928A05109297
:106560008905109288054981442309F0BAC18091B8
:106570008D05882309F0B5C18091A2092090A2055C
:106580003090A305E090B0088090260990902709EC
:106590004090390950903A098F3F09F4BFC0FF2459
:1065A00000E010E0A82EBB24A7FCB094CB2CDB2C81
:1065B0006A817B818C819D81A80197010E94914B0A
:1065C000C401AA2797FDA095BA2F281B390B4A0BA7
:1065D0005B0BCA01B901A60195010E941D4B20E089
:1065E00032E040E050E00E94914B39014A01688559
:1065F00079858A859B85A80197010E94914BC201EC
:10660000AA2797FDA095BA2F281B390B4A0B5B0BC5
:10661000CA01B901A60195010E941D4B20E032E09C
:1066200040E050E00E94914B79018A0151E4251627
:1066300031043CF48091A4059091A5058134910525
:10664000A4F0C401B30122E030E040E050E00E9439
:10665000914B39014A01C801B70122E030E040E026
:1066600050E00E94914B79018A01E0919F08F0E08F
:10667000EE0FFF1FE259F74F0190F081E02DF7FF79
:1066800003C0F095E195FF4F7A97A4F0C401B301E0
:1066900023E030E040E050E00E94914B39014A0194
:1066A000C801B70123E030E040E050E00E94914B88
:1066B00079018A018091A409A82EBB24A7FCB0947B
:1066C000CB2CDB2CA4019301A614B704C804D90475
:1066D00014F4A6019501992787FD909590958195D1
:1066E0009F4FAA2797FDA095BA2F39014A01281775
:1066F00039074A075B0714F43C014D01AE14BF048F
:10670000C006D10614F486017501E816F9060A07D9
:106710001B070CF0BEC07C018D01BBC0FF2400E054
:1067200010E06A817B818C819D81A80197010E9484
:10673000914B59016A01C401AA2797FDA095BA2F70
:10674000A81AB90ACA0ADB0A688579858A859B85F1
:10675000A80197010E94914B79018A01C201AA27E1
:1067600097FDA095BA2FE81AF90A0A0B1B0BC60170
:10677000B50120E130E040E050E00E94914B39014A
:106780004A01C801B70120E130E040E050E00E943A
:10679000914B79018A0161E4261631043CF4809121
:1067A000A4059091A50581349105A4F0C401B3011D
:1067B00023E030E040E050E00E94914B39014A0173
:1067C000C801B70123E030E040E050E00E94914B67
:1067D00079018A01E0919F08F0E0EE0FFF1FE25976
:1067E000F74F0190F081E02DF7FF03C0F095E195A0
:1067F000FF4F7A97A4F0C401B30123E030E040E0FA
:1068000050E00E94914B39014A01C801B70123E0D1
:1068100030E040E050E00E94914B79018A0171E242
:10682000671671048104910434F090E2692E712C92
:10683000812C912C11C080EE68168FEF78068FEFB7
:1068400088068FEF980644F480EE682E8FEF782E3E
:106850008FEF882E8FEF982E91E2E916F104010553
:10686000110534F010E2E12EF12C012D112D11C093
:10687000A0EEEA16AFEFFA06AFEF0A07AFEF1A077E
:1068800044F4B0EEEB2EBFEFFB2EBFEF0B2FBFEFAC
:106890001B2F80914B0590914C05A0914D05B09117
:1068A0004E0586199709A809B90980934B0590935D
:1068B0004C05A0934D05B0934E05809153059091E2
:1068C0005405A0915505B09156058E199F09A00B4E
:1068D000B10B8093530590935405A0935505B09345
:1068E00056058091FA049091FB048F3F910509F0C1
:1068F00008F4E1C4B981BB2309F05FC480918D0520
:10690000882309F05AC480916F05882309F055C483
:1069100060910E0970910F098091100990911109F1
:1069200020E031E040E050E00E94914B19012A0143
:1069300020930E0930930F094093100950931109C9
:1069400060911509709116098091170990911809A5
:1069500020E031E040E050E00E94914B288F398FD9
:106960004A8F5B8F209315093093160940931709BE
:1069700050931809E090B008FF2400E010E0209147
:106980003B0530913C0540913D0550913E05C801C5
:10699000B7010E941D4B20E031E040E050E00E9432
:1069A000914B59016A0120933B0530933C0540937C
:1069B0003D0550933E0520913F05309140054091A3
:1069C000410550914205C801B7010E941D4B20E0CE
:1069D00031E040E050E00E94914B39014A012093A0
:1069E0003F05309340054093410550934205609127
:1069F000430570914405809145059091460520E03E
:106A000031E040E050E00E94914B209343053093E9
:106A100044054093450550934605E090C908FF247E
:106A200000E010E0C201B1016A197B098C099D09DF
:106A3000A80197010E94914B2093C3053093C40590
:106A40004093C5055093C605CA01B90120E031E065
:106A500040E050E00E94914B690130938B052093F8
:106A60008A05688D798D8A8D9B8D661977098809CD
:106A70009909A80197010E94914BCA01B90120E030
:106A800031E040E050E00E94914B8901309389054C
:106A9000209388058091A2059091A30581349105EA
:106AA000C4F48091A4059091A505813491058CF4DE
:106AB000E0919F08F0E0EE0FFF1FE259F74F0190C1
:106AC000F081E02DF7FF03C0F095E195FF4F7A9735
:106AD000B4F08091A2098F3F91F4C60162E070E0AA
:106AE0000E945C4B70938B0560938A05C80162E03D
:106AF00070E00E945C4B70938905609388056091FB
:106B0000060970910709809108099091090920E010
:106B100031E040E050E00E94914B20930609309311
:106B2000070940930809509309096091FB08709187
:106B3000FC088091FD089091FE0820E031E040E0E3
:106B400050E00E94914B2093FB083093FC08409347
:106B5000FD085093FE08E8A0F9A00AA11BA12A8114
:106B60003B814C815D81E21AF30A040B150BE09224
:106B7000DA05F092DB050093DC051093DD05AC8CA3
:106B8000BD8CCE8CDF8C488559856A857B85A41A9F
:106B9000B50AC60AD70AA092D605B092D705C09208
:106BA000D805D092D905E092D205F092D305009392
:106BB000D4051093D505A092CE05B092CF05C09212
:106BC000D005D092D10580914F0590915005A091AC
:106BD0005105B09152058E199F09A00BB10B8093FE
:106BE0004F0590935005A0935105B09352058091A5
:106BF000570590915805A0915905B0915A058A19E9
:106C00009B09AC09BD098093570590935805A09343
:106C10005905B0935A0520917005309171052138BE
:106C2000310594F08091190590911A050196909381
:106C30001A05809319058091190990911A090196F6
:106C400090931A098093190920583F4F94F480912A
:106C5000190590911A05019790931A0580931905CB
:106C60008091190990911A09019790931A098093BC
:106C70001909688D798D8A8D9B8D2AE130E040E07D
:106C800050E00E94914B30933F0820933E081092B1
:106C900071051092700581E090E09093B6058093A5
:106CA000B5058091AD059091AE05A091AF05B0916D
:106CB000B00582199309A409B509815E914BAF4FC4
:106CC000BF4F8F539C49A040B04028F08091A3094A
:106CD00081330CF4C1C071E0E71670E1F70670E093
:106CE000070770E017070CF452C08091B4058823A1
:106CF00009F449C0D801C7017CE0B595A7959795DF
:106D000087957A95D1F701969093B6058093B5054E
:106D1000D801C70163E0B595A795979587956A95C2
:106D2000D1F78093C3059093C405A093C505B09394
:106D3000C60589589341A040B04064F088E893E1CB
:106D4000A0E0B0E08093C3059093C405A093C5056F
:106D5000B093C6056091C3057091C4058091C505C7
:106D60009091C60520E031E040E050E00E94914B58
:106D700080918A0590918B05820F931F90938B05CC
:106D800080938A0566C081E08093B40562C010924A
:106D9000B405F0E0EF16F0EFFF06FFEF0F07FFEF8F
:106DA0001F070CF056C08091B305882309F44DC02D
:106DB00088279927DC018E199F09A00BB10B5CE095
:106DC000B595A795979587955A95D1F70196909384
:106DD000B6058093B505C801B70128E030E040E072
:106DE00050E00E94914B2093C3053093C40540931B
:106DF000C5055093C60528573C4E4F4F5F4F64F46E
:106E000088E79CEEAFEFBFEF8093C3059093C40576
:106E1000A093C505B093C6056091C3057091C405E4
:106E20008091C5059091C60520E031E040E050E03A
:106E30000E94914B80918A0590918B05820F931F40
:106E400090938B0580938A0511C081E08093B305F0
:106E50000DC01092B3050AC01092B6051092B50588
:106E600088EE93E090939403809393038091CA08F3
:106E7000482E55248091B5059091B60548165906BF
:106E800024F45092B6054092B5059090A309692C60
:106E9000772467FC70948091B5059091B60544E025
:106EA000880F991F4A95E1F76816790674F4892DC1
:106EB00097FC815F8595859585958595992787FDB3
:106EC00090959093B6058093B50571E0E71674E050
:106ED000F70670E0070770E0170774F0809115055A
:106EE000909116052091B5053091B605820F931F3C
:106EF000909316058093150580E0E8168CEFF80650
:106F00008FEF08078FEF180774F4809115059091A3
:106F100016052091B5053091B605821B930B909311
:106F200016058093150581E090E09093B605809357
:106F3000B5051092BF051092C0051092C1051092C0
:106F4000C2058091A9059091AA05A091AB05B091C9
:106F5000AC05288D398D4A8D5B8D821B930BA40B5C
:106F6000B50B815E914BAF4FBF4F8F539C49A040F3
:106F7000B04020F040E349150CF0C1C051E0A51627
:106F800050E1B50650E0C50650E0D5060CF452C0FD
:106F90008091B205882309F449C0D601C5013CE0BF
:106FA000B595A795979587953A95D1F701969093C2
:106FB000B6058093B505D601C50123E0B595A79523
:106FC000979587952A95D1F78093BF059093C00533
:106FD000A093C105B093C20589589341A040B04029
:106FE00064F088E893E1A0E0B0E08093BF0590935F
:106FF000C005A093C105B093C2056091BF05709113
:10700000C0058091C1059091C20520E031E040E0CB
:1070100050E00E94914B8091880590918905820FE4
:10702000931F909389058093880566C081E08093C3
:10703000B20562C01092B20570E0A71670EFB706F5
:107040007FEFC7067FEFD7060CF056C08091B105E1
:10705000882309F44DC088279927DC018A199B09E8
:10706000AC09BD090CE0B595A795979587950A954C
:10707000D1F701969093B6058093B505C601B50189
:1070800028E030E040E050E00E94914B2093BF05A3
:107090003093C0054093C1055093C20528573C4E1C
:1070A0004F4F5F4F64F488E79CEEAFEFBFEF8093E4
:1070B000BF059093C005A093C105B093C205609130
:1070C000BF057091C0058091C1059091C20520E077
:1070D00031E040E050E00E94914B80918805909112
:1070E0008905820F931F909389058093880511C0AD
:1070F00081E08093B1050DC01092B1050AC01092D5
:10710000B6051092B50588EE93E0909394038093B2
:1071100093038091B5059091B6054816590624F45D
:107120005092B6054092B5058091B5059091B6058F
:1071300014E0880F991F1A95E1F76816790674F420
:10714000892D97FC815F85958595859585959927EE
:1071500087FD90959093B6058093B50591E0A916AB
:1071600094E0B90690E0C90690E0D90674F08091E9
:107170001705909118052091B5053091B605820F3D
:10718000931F9093180580931705A0E0AA16ACEF03
:10719000BA06AFEFCA06AFEFDA06CCF48091170556
:1071A000909118052091B5053091B605821B930B7F
:1071B00090931805809317050AC0109289051092C4
:1071C000880510928B0510928A0510926F0520E0B9
:1071D00030E040E050E060911B0970911C09809103
:1071E0001D0990911E090E943D4A882341F4109286
:1071F00089051092880510928B0510928A0580915E
:107200000E0990910F09A0911009B0911109809376
:10721000AD059093AE05A093AF05B093B0058091F6
:10722000150990911609A0911709B091180980933A
:10723000A9059093AA05A093AB05B093AC05109255
:107240003B0510923C0510923D0510923E051092B0
:107250003F05109240051092410510924205109290
:107260004305109244051092450510924605109270
:107270000E0910920F091092100910921109109224
:1072800015091092160910921709109218091092F8
:107290000609109207091092080910920909109224
:1072A000FB081092FC081092FD081092FE08109244
:1072B000FB041092FA04C0907F05D09080058601EF
:1072C000D7FE04C0002711270C191D090031110534
:1072D0006CF088EE93E090939403809393038091F5
:1072E000A40884FD03C081E08093C705E090AD0849
:1072F000B601882777FD8095982F2E2D30E040E04D
:1073000050E00E941D4B9801442737FD4095542FB3
:107310000E941D4B20E032E040E050E00E94914B83
:1073200089019A01FF24EC9CC001ED9C900DFC9C0E
:10733000900D112464E070E00E945C4B600F711F9F
:10734000882777FD8095982F6093DE057093DF0581
:107350008093E0059093E10520915B0530915C05F9
:1073600040915D0550915E05261B370B480B590B6C
:1073700020935B0530935C0540935D0550935E055B
:107380002155334C4040504064F080E593ECA0E040
:10739000B0E080935B0590935C05A0935D05B0938E
:1073A0005E0580915B0590915C05A0915D05B091B3
:1073B0005E05805B9C43AF4FBF4F64F480EB9CE362
:1073C000AFEFBFEF80935B0590935C05A0935D05E5
:1073D000B0935E058091670590916805892B09F44B
:1073E00056C18091A40883FF52C16A817B818C8140
:1073F0009D8120E032E040E050E00E94914B890105
:1074000037FF03C0109501951F4F688579858A85E0
:107410009B8520E032E040E050E00E94914B290142
:1074200037FF04C0509441945108539440165106BC
:107430000CF42801209167053091680560913509A9
:10744000709136098091370990913809B090C7053D
:10745000BB2001F5245E3D4F79010027F7FC009524
:10746000102F2BE035E040E050E00E94914BE21AF3
:10747000F30A040B150BC801B70128E631E040E020
:1074800050E00E94914BBCE4EB2EBFEFFB2EE60ECA
:10749000F71E18C06091670570916805882777FD11
:1074A0008095982F2BE035E040E050E00E941D4B86
:1074B00060933509709336098093370990933809A2
:1074C000EE24FF24C0909303D0909403C114D10400
:1074D00051F5F9E14F16510434F580917005909102
:1074E00071058E0D9F1D9093710580937005BB20D3
:1074F000D1F088EC90E09093DE048093DD046091FD
:1075000035097091360980913709909138092BE03F
:1075100035E040E050E00E94914B30936A052093A3
:1075200069051092C705009135091091360920911F
:10753000370930913809C20168E070E00E945C4B65
:107540006F5F7F4FC701A3E0880F991FAA95E1F7EE
:107550000E945C4B4B01AA2497FCA094BA2C800E8D
:10756000911EA21EB31E8092350990923609A092F8
:107570003709B09238098091A503682E7724469C7C
:10758000C001479C900D569C900D112460E270E064
:107590000E945C4B2301461A570A57FC72C0C11463
:1075A000D10409F01EC58091A4059091A5052091F4
:1075B000A2053091A305820F931F68E070E00E943E
:1075C0005C4B6B0120E430E0C20ED31E8091690554
:1075D00090916A05AA2797FDA095BA2FFCE1EF2E9E
:1075E000F2E0FF2E012D112DE81AF90A0A0B1B0BF0
:1075F000C501B4012BE035E040E050E00E94914B22
:10760000E20EF31E041F151FC801B70128E631E082
:1076100040E050E00E94914B645B7040649DC0016B
:10762000659D900D749D900D1124B6010E945C4BD8
:107630009301220F331F260D371D2617370734F00D
:10764000309521953F4F621773070CF4B9019B01E8
:10765000442737FD4095542F80915B0590915C0540
:10766000A0915D05B0915E05820F931FA41FB51F09
:1076700080935B0590935C05A0935D05B0935E05D8
:1076800006C084EF91E090939403809393038091DC
:10769000C80581508093C8058F3F09F09AC088E1E2
:1076A0008093C805E090B008FF2400E010E06A81F4
:1076B0007B818C819D81A80197010E94914B309321
:1076C000130820931208688579858A859B85A8010F
:1076D00097010E94914B30931508209314088091D4
:1076E0002609909127099093170880931608809196
:1076F000390990913A09909319088093180880915C
:107700002B0990912C0990931B0880931A08809163
:1077100084059091850590931D0880931C086091C5
:10772000630570916405809165059091660520E080
:1077300032E040E050E00E94914B30931F082093CC
:107740001E088091670590916805909323088093A7
:107750002208809111039091120390932508809341
:10776000240860913509709136098091370990910C
:1077700038092BE035E040E050E00E94914B309317
:1077800029082093280880917A0590E09093270893
:10779000809326088091A0099091A10990933508C3
:1077A0008093340880919E0990919F0990933708A7
:1077B0008093360880916B0790E09093390880930E
:1077C00038088091E0049091E10490933B08809305
:1077D0003A0839813323A9F06091010970910209B7
:1077E000882777FD8095982F0E94024A20913009C2
:1077F0003091310940913209509133090E94BA4ABF
:107800002EC0E0900109F09002096A817B818C8191
:107810009D810E94024A20911B0930911C094091D0
:107820001D0950911E090E94BA4A5B016C01002794
:10783000F7FC0095102FC801B7010E94024A209161
:1078400030093091310940913209509133090E9439
:10785000BA4A9B01AC01C601B5010E9403490E94CE
:10786000CF49709302096093010980918D058823A7
:10787000A9F06091F5087091F608882777FD80954A
:10788000982F0E94024A209130093091310940918D
:107890003209509133090E94BA4A2EC0E090F5088F
:1078A000F090F608688579858A859B850E94024A52
:1078B00020911B0930911C0940911D0950911E090E
:1078C0000E94BA4A5B016C010027F7FC0095102F5B
:1078D000C801B7010E94024A209130093091310954
:1078E00040913209509133090E94BA4A9B01AC0180
:1078F000C601B5010E9403490E94CF497093F60862
:107900006093F50860912B0970912C09882777FD09
:107910008095982F0E94024A7B018C01609130096A
:107920007091310980913209909133099B01AC012A
:107930000E9403499B01AC01C801B7010E94BA4AE9
:107940007B018C0160914705709148058091490544
:1079500090914A050E94024A20911B0930911C090E
:1079600040911D0950911E090E94BA4A20E030E062
:1079700040E05FE30E94BA4A9B01AC01C801B70135
:107980000E9403490E94CF4970932C0960932B09F0
:10799000809101099091020990933D0880933C08E1
:1079A0008091F5089091F60890933F0880933E08E7
:1079B00080910109909102098150904434F080E057
:1079C00090E49093020980930109809101099091BC
:1079D00002098050904C34F480E090EC90930209BE
:1079E000809301098091F5089091F60881509044A8
:1079F00034F080E090E49093F6088093F50880914D
:107A0000F5089091F6088050904C34F480E090ECAA
:107A10009093F6088093F50880912B0990912C099A
:107A20008150904434F080E090E490932C0980934E
:107A30002B0980912B0990912C098050904C34F4A3
:107A400080E090EC90932C0980932B09EC85FD85C8
:107A5000EE0FFF1FEE0FFF1FFD87EC870E94D8453A
:107A600020910409422F50E05F8B4E8B2C853D8581
:107A7000281B390B241735070CF49A0180912A0929
:107A8000682F70E07D8B6C8B8B01000F111F000F36
:107A9000111FC801805590403DA32CA38217930766
:107AA00014F49DA38CA38CA19DA190932108809395
:107AB000200860912B0970912C098091DE0590912E
:107AC000DF05A091E005B091E10522E0880F991F44
:107AD000AA1FBB1F2A95D1F7681B790BACA1BDA1CA
:107AE000A03AB1055CF4A69FC001A79F900DB69F78
:107AF000900D112460EA70E00E945C4B8CA19DA166
:107B000095958795861797070CF4BC0190958195FC
:107B10009F4F681779070CF4BC01C801ECA1FDA1C7
:107B20008E1B9F0B861797070CF4BC018CA19DA19F
:107B3000801B910B1B01681779070CF41C018091C5
:107B400001099091020980907B0590907C0588192D
:107B5000990990930D0980930C0940901B0950904E
:107B60001C0960901D0970901E0920E030E040E083
:107B700050E0C301B2010E943D4A8823D1F16091D7
:107B8000E6057091E7058091E8059091E9050E946E
:107B9000024A5B016C0160912B0570912C0580916C
:107BA0002D0590912E050E94024AA30192010E9488
:107BB000BA4A7B018C01B401882777FD8095982F04
:107BC0000E94024A9B01AC01C801B7010E94024910
:107BD0009B01AC01C601B5010E9403490E94CF4937
:107BE0006093E6057093E7058093E8059093E905B7
:107BF0001CC020910C0930910D09442737FD409598
:107C0000542F8091E6059091E705A091E805B09189
:107C1000E905820F931FA41FB51F8093E60590937B
:107C2000E705A093E805B093E9058091E6059091FA
:107C3000E705A091E805B091E90581509A4FA04071
:107C4000B04064F080E09AEFA0E0B0E08093E605F9
:107C50009093E705A093E805B093E9058091E605C8
:107C60009091E705A091E805B091E9058050964014
:107C7000AF4FBF4F64F480E096E0AFEFBFEF80936B
:107C8000E6059093E705A093E805B093E9056091B8
:107C90000C0970910D0980919D0390919E03A09114
:107CA0009F03B091A003888B998BAA8BBB8B8827ED
:107CB00077FD8095982F0E94024A7B018C0160918C
:107CC000E6057091E7058091E8059091E9050E942D
:107CD000024A9B01AC01688979898A899B890E9443
:107CE000BA4A9B01AC01C801B7010E9403490E9436
:107CF000CF497B018C016B01C10137FE04C088278D
:107D000099278219930962E070E00E945C4BACA154
:107D1000BDA16A0F7B1F882777FD8095982F209142
:107D2000AC0330E040E050E00E941D4B20E430E026
:107D300040E050E00E94914B3F832E83C216D30651
:107D40000CF497014E815F81509541955F4F5F879D
:107D50004E87241735070CF49A010CA11DA1020DC2
:107D6000131DC801820F931F64E070E00E945C4BFA
:107D700077FF03C060E070E006C08C899D8986179C
:107D800097070CF4BC01AE89BF896A177B070CF416
:107D9000BD016093F708C801821B930B64E070E09B
:107DA0000E945C4B77FF03C060E070E006C0EC8986
:107DB000FD89E617F7070CF4BF012E893F8962178A
:107DC00073070CF4B901609300098091F508909154
:107DD000F60880907D0590907E058819990990930A
:107DE000F4088093F30820E030E040E050E0C30165
:107DF000B2010E943D4A8823D1F16091E205709161
:107E0000E3058091E4059091E5050E94024A5B013B
:107E10006C01609133057091340580913505909126
:107E200036050E94024AA30192010E94BA4A7B01D0
:107E30008C01B401882777FD8095982F0E94024A13
:107E40009B01AC01C801B7010E9402499B01AC0132
:107E5000C601B5010E9403490E94CF496093E20523
:107E60007093E3058093E4059093E5051CC0209191
:107E7000F3083091F408442737FD4095542F809142
:107E8000E2059091E305A091E405B091E505820F2C
:107E9000931FA41FB51F8093E2059093E305A09361
:107EA000E405B093E5058091E2059091E305A0918A
:107EB000E405B091E50581509A4FA040B04064F0D0
:107EC00080E09AEFA0E0B0E08093E2059093E305B4
:107ED000A093E405B093E5058091E2059091E30558
:107EE000A091E405B091E50580509640AF4FBF4F9B
:107EF00064F480E096E0AFEFBFEF8093E2059093EB
:107F0000E305A093E405B093E5056091F308709153
:107F1000F408882777FD8095982F0E94024A7B01FC
:107F20008C016091E2057091E3058091E4059091E8
:107F3000E5050E94024A9B01AC01688979898A891A
:107F40009B890E94BA4A9B01AC01C801B7010E94FB
:107F500003490E94CF492E813F81621773070CF4B9
:107F60009B010E851F85021713070CF489018CA154
:107F70009DA182199309800F911F64E070E00E9417
:107F80005C4B77FF03C060E070E006C08C899D8980
:107F9000861797070CF4BC01AE89BF896A177B0767
:107FA0000CF4BD0160932209ECA1FDA1E01BF10BD3
:107FB000CF018219930964E070E00E945C4B77FF67
:107FC00003C060E070E006C02C893D8926173707A2
:107FD0000CF4B9014E895F896417750754F4BA012E
:107FE00008C00894C108D108D0929403C0929303AA
:107FF0004ECB60931F09A5960FB6F894DEBF0FBE57
:10800000CDBFDF91CF911F910F91FF90EF90DF9047
:10801000CF90BF90AF909F908F907F906F905F9028
:108020004F903F902F90089584B1806A84B93D9A13
:1080300082E58CBD1DBC459A91E090933F098AEA88
:108040008093430983E8809344098AE0809345093B
:108050001092470910924609109249091092480956
:108060001092650990936609809367099093680957
:1080700083E0809369090895F89460912B057091CD
:108080002C0580912D0590912E052CE630E040E0E6
:1080900050E00E94914B309347092093460960912C
:1080A00033057091340580913505909136052CE6A5
:1080B00030E040E050E00E94914B3093490920931A
:1080C000480960913509709136098091370990917E
:1080D00038092BE035E040E050E00E94914B3093AE
:1080E0004F0920934E09209123053091240580915A
:1080F000120990911309B9010E945C4BCB01880FC2
:10810000991F860F971F880F991F880F991F9093AB
:108110004B0980934A0980912E0990912F09B9014A
:108120000E945C4BCB01880F991F860F971F880F09
:10813000991F880F991F90934D0980934C091092B5
:10814000240510922305109213091092120910921F
:108150002F0910922E09809145098C3009F4E7C04F
:108160008D3030F48A3051F08B3009F002C16EC08E
:108170008D30D9F18E3009F0FCC0EBC080919205B2
:1081800080935609809193058093570980919405B7
:10819000809358098091950580935909809196059F
:1081A00080935A098091970580935B098091980587
:1081B00080935C098091990580935D098091A80561
:1081C00080935E09837F8093A8058091110390912D
:1081D000120380935F098091B40880936009A2E044
:1081E000B0E00E94E34B802D2EC08091D408809394
:1081F00056098091D508809357098091D6088093BD
:1082000058098091D708809359098091D8088093A4
:108210005A098091D90880935B098091DA0880938C
:108220005C098091DB0880935D098091DE08809372
:108230005E098091DC0880935F098091DD0880935E
:1082400060098091DF088093610993C0E0919E08E6
:10825000F0E0EE0FFF1FE259F74F0190F081E02DA3
:108260002FEFE138F20714F4E1E8FFEFE038F10511
:1082700014F0EFE7F0E0E0935609E0919F08F0E09A
:10828000EE0FFF1FE259F74F0190F081E02D6FEFE5
:10829000E138F60714F4E1E8FFEFE038F10514F0F7
:1082A000EFE7F0E0E0935709E0919D08F0E0EE0F72
:1082B000FF1FE259F74F0190F081E02D8FEFE13879
:1082C000F80714F4E1E8FFEFE038F10514F0EFE708
:1082D000F0E0E0935809E0919C08F0E0EE0FFF1FFA
:1082E000E259F74F0190F081E02D2FEFE138F207CE
:1082F00014F4E1E8FFEFE038F10514F0EFE7F0E007
:10830000E09359098091720580935A098091740510
:1083100080935B098091760580935C098091780554
:1083200080935D0980917A0580935E0922C08091D7
:108330006B07863018F010926B0785E08093560922
:1083400080918405909185059093590980935809EF
:1083500010C08091660980935609809167098093C7
:108360005709809168098093580980916909809321
:108370005909789480916509882309F478C040915F
:108380006B0950916C09CA0181509E4F8F5F9340D9
:10839000B0F420916D0930916E09C90181509E4F52
:1083A0008F5F934060F48091A40885FF08C05093CC
:1083B00016064093150630931806209317068091F1
:1083C00071099091720921E08936920724F4909303
:1083D00068058093670580916705909168052091F5
:1083E000690530916A05845E9D4F821B930B68E698
:1083F00071E00E945C4B845B904090936C0580938D
:108400006B0520917509309176098091DD0490917A
:10841000DE048217930740F480916B07882321F4D0
:108420003093DE042093DD0480916A09843679F06C
:10843000873629F5809177098093A2098091780980
:108440008093A409809179098093A309089580916C
:10845000770990E090939F0980939E098091790914
:1084600090917A099093A1098093A00908951092A0
:108470001606109215061092180610921706089507
:1084800080913F09882309F43BC0459883E499E033
:1084900090934109809340099091F205E92FF0E013
:1084A000E155FC4F8081809345099F5F9093F205D1
:1084B000963010F01092F20510923F090E943C4055
:1084C00081E08093420900000000000000000000ED
:1084D000000000000000000000000000000000009C
:1084E000000000000000000000000000000000008C
:1084F00000000000000080914309809362098EBD56
:10850000089580913F09882309F07CC00DB407FECF
:1085100079C084E08093DF04459A2EB58091F405FC
:10852000813069F0813018F08230C9F513C01092A3
:1085300064092093F305213891F581E008C02535C1
:1085400041F58091F3058B5A8093F30582E0809387
:10855000F40525C080916409E82FF0E0EC57F64F50
:1085600020838F5F809364099091F3058A31A0F096
:10857000291769F4AAE6B9E0E4E8F9E08AE1019094
:108580000D928150E1F781E08093650902C010925D
:1085900065091092F40503C0920F9093F3052091A2
:1085A0004209203208F028C0459800000000000071
:1085B00000000000000000000000000000000000BB
:1085C00000000000000000000000000000000000AB
:1085D00000000000000000000000E0914009F09160
:1085E0004109E20FF11D80818EBD80819091620969
:1085F000890F8093620903C081E080933F092F5F58
:10860000209342090895982F8091CD0881FF05C0DD
:1086100080E0992309F481E0982F992331F080912B
:10862000FC05882311F0429A089542980895982FE6
:108630008091CD0881FF05C080E0992309F481E095
:10864000982F992331F08091FC05882311F0439AEB
:1086500008954398089587B18C6087B980E00E949F
:10866000034380E00E9417431092F90580E880934D
:10867000B5031092FA058093B603089540918305DF
:10868000442389F58091CF0883FF2AC080919E08FA
:10869000E82FF0E0EE0FFF1FE259F74F8081918144
:1086A0008C5A9F4F04F18081918180359105DCF4D3
:1086B00080919F08E82FF0E0EE0FFF1FE259F74F7F
:1086C00080819181855B9F4F1CF481E08093FB0545
:1086D000808191818C34910534F01092FB0503C0A8
:1086E00081E08093FB058091CF08282F82FF02C094
:1086F0004093FB058091FB058093FC058091FD056F
:1087000081508093FD058F3F09F082C084E0809303
:10871000FD0524FF19C020911103309112038091AF
:10872000B40890E0281739077CF48091CD08282FF1
:1087300080FF03C081E08093FC0522FF02C081E03E
:1087400001C082E08093FD058091D1088B3F88F0C5
:1087500080911409873E20F08091D008807823C052
:108760008A3038F490E08091D00887FF91E0892F1B
:108770001AC08091F90581508093F9058F3FA9F4C3
:108780008091140981508093F9058091B50381305F
:1087900011F480E801C086958093B5038091D008DC
:1087A0009091B50389230E9403438091D3088B3FA6
:1087B00098F080912909873E20F08091D208807836
:1087C00008C08A3048F490E08091D20887FF91E099
:1087D000892F0E94174308958091FA058150809354
:1087E000FA058F3FA9F48091290981508093FA05F9
:1087F0008091B603813011F480E801C086958093A2
:10880000B6038091D2089091B60389230E94174342
:108810000895EF92FF920F931F93CF93DF93809170
:108820008305882309F469C1E090FE05F090FF05F7
:10883000F0920106E092000680919E08C82FD0E0D9
:10884000FE01EE0FFF1FE259F74F0190F081E02D7E
:108850008091020690910306E81BF90BF093A6099C
:10886000E093A509EE9FC001EF9F900DFE9F900D34
:1088700011241E161F063CF466E970E00E945C4B52
:10888000E60FF71F06C066E970E00E945C4BE61B2E
:10889000F70BF093A609E093A509C701880F991F6C
:1088A0002091A5093091A609820F931F63E070E023
:1088B0000E945C4B9B017093FF056093FE05E09165
:1088C0000406F09105068B010E0F1F1F809106060E
:1088D000853009F45EC0863048F4833079F1843005
:1088E00008F04EC0823009F038C10AC0873009F460
:1088F000AAC0873008F48EC0883009F02EC1D3C0DA
:1089000046E0E416F1040CF428C1C701861B970B5E
:108910009C018091B90890E0281739070CF41DC11B
:10892000F0920506E092040683E08093060689E152
:1089300090E09093B9038093B8030FC18091B8037E
:108940009091B90301979093B9038093B803892B51
:1089500039F4109205061092040682E08093060610
:108960002B5F3F4F2B30310548F48091A40880FFE6
:1089700002C087E001C084E0809306068F01EDC04D
:108980008091BA0890E0081719070CF0E6C08C0136
:10899000E4C08091CF0886FF28C0CC0FDD1FC259EC
:1089A000D74F888199818C5A9F4F3CF084E690E0A4
:1089B0009093B9038093B80318C08091B803909145
:1089C000B90301979093B9038093B803892B69F495
:1089D00082E080930606109205061092040684EF4A
:1089E00091E09093DE048093DD048091BA0890E0DA
:1089F000081719070CF48C012C5F3F4F2930310503
:108A000008F0ABC089E190E09093B9038093B8037C
:108A100086E016C0CB010496099788F4E616F7069F
:108A200071F48091B8039091B90301979093B903C1
:108A30008093B803892B09F090C087E001C085E0DE
:108A4000809306068AC08091FF0490910005909360
:108A50000806809307066091630570916405809114
:108A600065059091660520E830E040E050E00E9406
:108A7000914B30930A062093090610920C0610922F
:108A80000B0610920E0610920D0610921006109210
:108A90000F061092110610921206109213061092F1
:108AA000140688E021C0CB0177FF04C088279927EE
:108AB000861B970B06970CF450C080910F0690917F
:108AC000100664E070E00E945C4BCF01861B970BA0
:108AD00090930506809304068901080F191F1092D0
:108AE0000E0610920D0685E08093060684EF91E055
:108AF0009093DE048093DD0430C0809106068823C5
:108B000019F08130E9F409C08091B7038150809356
:108B1000B7038F3F01F581E01CC0E0919E08F0E0B3
:108B2000EE0FFF1FE259F74F80819181909303066A
:108B300080930206855B9F4F5CF41092BA0308C0D5
:108B400010920506109204061092FF051092FE0581
:108B500082E08093060600E010E080910406909188
:108B6000050697FF04C010920506109204069801AE
:108B700017FF02C020E030E08091FE059091FF05D4
:108B8000909347088093460830934B0820934A08F7
:108B9000809104069091050690934D0880934C08AF
:108BA000C901DF91CF911F910F91FF90EF90089530
:108BB0009F92AF92BF92CF92DF92EF92FF920F936C
:108BC0001F93CF93DF9380910606883009F01EC172
:108BD00080916D05882309F019C1E090FF04F090A1
:108BE00000058091070690910806E81AF90A00919D
:108BF000A3038091BB0890E09C012E9DC0012F9D96
:108C0000900D3E9D900D112464E070E00E945C4B3D
:108C10009B01442737FD4095542F80911106909178
:108C20001206A0911306B0911406280F391F4A1F8F
:108C30005B1F209311063093120640931306509346
:108C40001406213462E436076FE0460760E05607F9
:108C50002CF080E492E4AFE0B0E009C0205C3D4B32
:108C6000404F5F4F64F480EC9DEBA0EFBFEF80932B
:108C7000110690931206A0931306B0931406A090C9
:108C80001106B0901206C0901306D0901406909072
:108C9000A103C0910B06D0910C0660916305709101
:108CA0006405809165059091660520E830E040E01C
:108CB00050E00E94914BCA01B90120910906309100
:108CC0000A06442737FD4095542F621B730B840B13
:108CD000950B2091A40330E040E050E00E941D4B32
:108CE00020E230E040E050E00E94914BC901309317
:108CF000A6092093A50921E0893192071CF088E19B
:108D000091E005C0885E9E4F34F488EE9EEF90930C
:108D1000A6098093A509802F90E0AC014E9DC0016B
:108D20004F9D900D5E9D900D112464E070E00E94B7
:108D30005C4B8B01C601B50120EA3FE040E050E00A
:108D40000E94914B020F131F97012C1B3D0B892D85
:108D500090E0BC01269FC001279F900D369F900D8B
:108D6000112462E070E00E945C4B8091A509909113
:108D7000A609680F791F600F711F8091A90890E004
:108D80009C01629FC001639F900D729F900D112402
:108D90006AE070E00E945C4B8091A70890E0880F29
:108DA000991F880F991F8617970714F4EC0109C0C3
:108DB00044275527481B590BEB01641775070CF422
:108DC000EA01D0930E06C0930D06F0920C06E092D5
:108DD0000B0620910F0630911006AE01421B530B7B
:108DE0008091BC0890E0BC01469FC001479F900D58
:108DF000569F900D112464E670E00E945C4B260F94
:108E0000371F3093100620930F0602C0C0E0D0E059
:108E100060911106709112068091130690911406CC
:108E200020EA3FE040E050E00E94914B30934F0831
:108E300020934E08D0934908C0934808CE01DF9193
:108E4000CF911F910F91FF90EF90DF90CF90BF9047
:108E5000AF909F90089580911D0690911E06A0915D
:108E60001F06B09120068093250690932606A093B6
:108E70002706B09328068091210690912206A091A2
:108E80002306B09124068093290690932A06A09386
:108E90002B06B0932C060895109216061092150614
:108EA00010921806109217060895A8E0B0E0EBE5BE
:108EB000F7E40C94B64B7B018C01611571058105BB
:108EC000910519F482E089835AC083E089838EE199
:108ED000C82ED12CDC82CB82ED82FE820F831887D4
:108EE000C801B7010E94C847BC016150704077FFBC
:108EF00033C0EE27FF27E61BF70B20E030E040E011
:108F000050E081E090E0A0E0B0E00E2E04C0880FB9
:108F1000991FAA1FBB1F0A94D2F70197A109B10993
:108F20008E219F21A023B1230097A105B10521F037
:108F300021E030E040E050E004C016950795F7943A
:108F4000E794EA95D2F72E293F29402B512B2D8308
:108F50003E834F8358870FC06115710581F0062E3F
:108F600004C0EE0CFF1C001F111F0A94D2F7ED8203
:108F7000FE820F831887C61AD70ADC82CB821A8238
:108F8000CE0101960E941548E8E028960C94D24B39
:108F9000EF92FF920F931F939B01AC01203080E072
:108FA000380781E0480780E0580780F42F3F3105FB
:108FB0004105510509F020F4EE24FF24870119C072
:108FC00068E0E62EF12C012D112D13C0203080E039
:108FD000380780E0480781E0580730F490E1E92E37
:108FE000F12C012D112D05C088E1E82EF12C012D69
:108FF000112D80E290E0A0E0B0E08E199F09A00B57
:10900000B10B04C05695479537952795EA94D2F74A
:10901000F901E554FC4F2081821B9109A109B10996
:109020001F910F91FF90EF9008959F92AF92BF9282
:10903000CF92DF92EF92FF920F931F93EE24FF24C3
:109040008701FC012481358146815781918080818F
:10905000823010F44061A2C0843009F49BC0823099
:1090600029F420E030E040E050E005C02115310552
:109070004105510519F4E0E0F0E092C0828193814E
:109080006FEF823896070CF05AC062E87FEF681BDA
:10909000790B6A3171052CF020E030E040E050E0BF
:1090A0002AC0AA24BB24650181E090E0A0E0B0E0E2
:1090B000062E04C0880F991FAA1FBB1F0A94D2F75F
:1090C0000197A109B10982239323A423B523009713
:1090D000A105B10529F071E0A72EB12CC12CD12C2E
:1090E00004C056954795379527956A95D2F72A2952
:1090F0003B294C295D29DA01C9018F779070A07056
:10910000B07080349105A105B10539F427FF09C07D
:10911000205C3F4F4F4F5F4F04C0215C3F4F4F4F8C
:109120005F4F80E090E0203060E0360760E0460767
:1091300060E4560710F081E090E0FC0123C0803825
:10914000910544F5FC01E158FF4FDA01C9018F7721
:109150009070A070B07080349105A105B10539F40C
:1091600027FF09C0205C3F4F4F4F5F4F04C0215C79
:109170003F4F4F4F5F4F57FF05C056954795379567
:109180002795319687E056954795379527958A9587
:10919000D1F706C020E030E040E050E0EFEFF0E033
:1091A000E22EF32E942F9F77802F8078892B9E2F8D
:1091B0009795992797958F77082F092B9E2F96952E
:1091C000812F8078892B9794992497948F77182FE3
:1091D0001929C801B7011F910F91FF90EF90DF90FF
:1091E000CF90BF90AF909F900895FC0141505040A8
:1091F00030F001900616D1F73197CF0108958827F6
:10920000992708955058BB27AA270ED079C16AD153
:1092100030F06FD120F031F49F3F11F41EF45FC1A4
:109220000EF4E095E7FB55C1E92F7BD180F3BA1727
:10923000620773078407950718F071F49EF593C1D0
:109240000EF4E0950B2EBA2FA02D0B01B901900161
:109250000C01CA01A0011124FF27591B99F0593FA5
:1092600050F4503E68F11A16F040A22F232F342FED
:109270004427585FF3CF469537952795A795F0403B
:109280005395C9F77EF41F16BA0B620B730B840B50
:10929000BAF09150A1F0FF0FBB1F661F771F881F08
:1092A000C2F70EC0BA0F621F731F841F48F4879560
:1092B00077956795B795F7959E3F08F0B3CF93954F
:1092C000880F08F09927EE0F9795879508950CD091
:1092D00017C10FD140F006D130F021F45F3F19F0F3
:1092E000F8C0511141C1FBC01CD198F39923C9F3B7
:1092F0005523B1F3951B550BBB27AA27621773079C
:10930000840738F09F5F5F4F220F331F441FAA1F4F
:10931000A9F333D00E2E3AF0E0E830D0915050400F
:10932000E695001CCAF729D0FE2F27D0660F771FBD
:10933000881FBB1F261737074807AB07B0E809F09F
:10934000BB0B802DBF01FF2793585F4F2AF09E3F34
:10935000510568F0BEC008C15F3FECF3983EDCF3F6
:10936000869577956795B795F7959F5FC9F7880FAD
:10937000911D9695879597F90895E1E0660F771FFF
:10938000881FBB1F621773078407BA0720F0621B90
:10939000730B840BBA0BEE1F88F7E095089504D089
:1093A0006894B111E1C00895C4D088F09F5790F03F
:1093B000B92F9927B751A0F0D1F0660F771F881FFA
:1093C000991F1AF0BA95C9F712C0B13081F0CBD00D
:1093D000B1E00895C8C0672F782F8827B85F39F0AB
:1093E000B93FCCF3869577956795B395D9F73EF459
:1093F00090958095709561957F4F8F4F9F4F089501
:10940000E89409C097FB3EF490958095709561951E
:109410007F4F8F4F9F4F9923A9F0F92F96E9BB27D4
:109420009395F695879577956795B795F111F8CF50
:10943000FAF4BB0F11F460FF1BC06F5F7F4F8F4FBB
:109440009F4F16C0882311F096E911C0772321F0B1
:109450009EE8872F762F05C0662371F096E8862F49
:1094600070E060E02AF09A95660F771F881FDAF7A0
:10947000880F9695879597F9089507D008F481E0AD
:10948000089503D008F48FEF0895990F0008550F41
:10949000AA0BE0E8FEEF16161706E807F907C0F07A
:1094A00012161306E407F50798F0621B730B840B82
:1094B000950B39F40A2661F0232B242B252B21F45C
:1094C00008950A2609F4A140A6958FEF811D811DFC
:1094D000089597F99F6780E870E060E008959FEF36
:1094E00080EC089500240A9416161706180609063B
:1094F000089500240A94121613061406050608950A
:10950000092E0394000C11F4882352F0BB0F40F491
:10951000BF2B11F460FF04C06F5F7F4F8F4F9F4FD1
:10952000089557FD9058440F551F59F05F3F71F053
:109530004795880F97FB991F61F09F3F79F08795BA
:109540000895121613061406551FF2CF4695F1DF43
:1095500008C0161617061806991FF1CF86957105D3
:10956000610508940895E894BB2766277727CB0107
:1095700097F908950BD0C4CFB5DF28F0BADF18F003
:10958000952309F0A6CFABCF1124EECFCADFA0F30D
:10959000959FD1F3950F50E0551F629FF001729F88
:1095A000BB27F00DB11D639FAA27F00DB11DAA1FA7
:1095B000649F6627B00DA11D661F829F2227B00DF4
:1095C000A11D621F739FB00DA11D621F839FA00D7F
:1095D000611D221F749F3327A00D611D231F849FCF
:1095E000600D211D822F762F6A2F11249F57504026
:1095F0008AF0E1F088234AF0EE0FFF1FBB1F661FC1
:10960000771F881F91505040A9F79E3F510570F079
:1096100060CFAACF5F3FECF3983EDCF38695779559
:109620006795B795F795E7959F5FC1F7FE2B880F74
:10963000911D9695879597F90895629FD001739F24
:10964000F001829FE00DF11D649FE00DF11D929FDE
:10965000F00D839FF00D749FF00D659FF00D99271D
:10966000729FB00DE11DF91F639FB00DE11DF91F41
:10967000BD01CF0111240895991B79E004C0991F01
:10968000961708F0961B881F7A95C9F7809508955C
:10969000AA1BBB1B51E107C0AA1FBB1FA617B70718
:1096A00010F0A61BB70B881F991F5A95A9F7809534
:1096B0009095BC01CD01089597FB092E07260AD08D
:1096C00077FD04D0E5DF06D000201AF4709561958F
:1096D0007F4F0895F6F7909581959F4F0895A1E2E9
:1096E0001A2EAA1BBB1BFD010DC0AA1FBB1FEE1F1C
:1096F000FF1FA217B307E407F50720F0A21BB30B67
:10970000E40BF50B661F771F881F991F1A9469F7E2
:1097100060957095809590959B01AC01BD01CF013E
:10972000089597FB092E05260ED057FD04D0D7DFEC
:109730000AD0001C38F450954095309521953F4F44
:109740004F4F5F4F0895F6F790958095709561950E
:109750007F4F8F4F9F4F08952F923F924F925F926E
:109760006F927F928F929F92AF92BF92CF92DF9231
:10977000EF92FF920F931F93CF93DF93CDB7DEB796
:10978000CA1BDB0B0FB6F894DEBF0FBECDBF09942A
:109790002A88398848885F846E847D848C849B8481
:1097A000AA84B984C884DF80EE80FD800C811B818F
:1097B000AA81B981CE0FD11D0FB6F894DEBF0FBEBE
:1097C000CDBFED010895F999FECFB2BDA1BDF89AC4
:1097D000119600B40895F999FECFB2BDA1BD00BCA9
:1097E00011960FB6F894FA9AF99A0FBE0895FFCF22
:1097F0000A010101FF6401C800496E746567726166
:109800006C4E69636B20202020496E74656772611D
:109810006C526F6C6C202020204163634E69636B37
:10982000202020202020202020416363526F6C6C78
:109830002020202020202020204779726F47696552
:10984000722020202020202020486F6568656E57F8
:109850006572742020202020204163635A2020203C
:10986000202020202020202020476173202020203D
:109870002020202020202020204B6F6D70617373EA
:1098800056616C7565202020205370616E6E756E78
:10989000672020202020202020456D7066616E67A3
:1098A00020202020202020202045727361747A6BB4
:1098B0006F6D706173732020204D6F746F725F56EF
:1098C0006F726E6520202020204D6F746F725F488C
:1098D000696E74656E202020204D6F746F725F4C2E
:1098E000696E6B7320202020204D6F746F725F5261
:1098F00065636874732020202020202020202020F1
:1099000020202020202020202044697374616E6371
:109910006520202020202020204F73644261722087
:109920002020202020202020204D4B334D61672017
:1099300043616C537461746520536572766F2020A7
:109940002020202020202020204E69636B20202012
:10995000202020202020202020526F6C6C202020EE
:1099600020202020202020202020202020202020F7
:1099700020202020202020202020202020202020E7
:1099800020202020202020202020202020202020D7
:10999000202020202020202020537469636B5661F2
:1099A0006C7565202020202020416C7469747564DA
:1099B00065204E2020202020205069746368436F6A
:1099C000756E7420202020202050697463684F66D3
:1099D000667365742020202020496E74656772616B
:1099E0006C416C7420202020204750535F526F6CD4
:1099F0006C20202020202020202800FFFF640080F1
:109A0000016400007D0000FF03737373010203040F
:109A100005060708090A48616C6C6F2057656C746D
:109A20000000000000000000000000000000000036
:109A30000000000000000000000000000000000026
:109A40000000000000000000000000000000000016
:109A50000000000000000000000000000000000006
:109A60000000000000000B01426567696E6E6572C0
:109A700000004E6F726D616C000053706F72740065
:109A8000006400F40190D0030090D0030017B7D118
:109A90003830FB103A409696020A644664ECFF0A9E
:109AA0000B0D0B0C0E01011919000100010202033C
:109AB0000303030404040404040404050505050564
:109AC0000505050505050505050505060606060641
:109AD0000606060606060606060606060606060626
:109AE0000606060606060606060606070707070711
:109AF00007070707070707070707070707070707F6
:109B000007070707070707070707070707070707E5
:109B100007070707070707070707070707070707D5
:109B200007070707070707070707070808080808C0
:109B300008080808080808080808080808080808A5
:109B40000808080808080808080808080808080895
:109B50000808080808080808080808080808080885
:109B60000808080808080808080808080808080875
:109B70000808080808080808080808080808080865
:109B80000808080808080808080808080808080855
:109B90000808080808080808080808080808080845
:0C9BA00008080808080808080808080061
:00000001FF
